:020000041100E9
:10300000002373B52B4D2C4C28006361022601F080
:1030100079F94021FE2221742800284B009601F006
:10302000C3F9002836D1217CFF222800244B0096CA
:1030300001F0BAF900282DD1224BA2899A4226D15B
:10304000E389214A93420DD1204B6361204B2268D2
:10305000002A03D1002B01D043CB43C4280001F048
:103060008FF973BD1B4A934201D00023EFE71A4B3F
:103070001A4A1B68934206D9C02304222800217CE7
:103080009B0001F007FA114B6361154BDFE700234A
:103090002374EAE7CC233821AC2228009B01217459
:1030A00001F0F8F90028F2D10E4B63610E4BE38179
:1030B0000E4BCCE7F441FF1F9C61FF1FA861FF1F6F
:1030C000AA61FF1F5959000083050000314100111A
:1030D00014BD001182150000C061FF1F871300009E
:1030E00020BD0011E9410011AAAAFFFF08BD00118F
:1030F000F7B5164B0192C318021D002000938823D8
:103100005B05D3181B685C1C1AD09CB2402C18D8E5
:103110008D781E0CAC466746CD782D023D43AE42FD
:1031200006D1019800280ED110000C70240A4C70B2
:1031300003249BB20733A343D218009B9A42DED3E9
:10314000FEBD4432F9E71000FAE7C046FC0F00006C
:10315000802213B503000324019189B25201073183
:103160009B18A14304305A1A88235B05C3181B68B7
:10317000591C03D190429241104016BD99B240298A
:1031800007D80B000733A343C0189042ECD30020AC
:10319000F3E74430F9E7134B134A1B68126810B584
:1031A000FA24934201D81A00F824104BE4021B6859
:1031B0009A4210D813000E4A12689A420ED3013375
:1031C00007D1F823DB029C4203D10A49054808F0E5
:1031D000AFFB200010BDFC24E402ECE7FE24E40277
:1031E000F7E7C04600C0071100D0071100E0071143
:1031F00000F00711FFFFFF7FF0B59BB015000490B2
:103200000391402A00D9A0E006AB59801A80FFF74D
:10321000C2FF0400042816D9002206A9FFF768FFA0
:10322000052810D906AB1B88AB420CD1002D07D066
:10323000514B2A000499C01808F02AFC002802D13A
:1032400001201BB0F0BD06AB1D8020000699FFF7E2
:103250007FFF041E7BD1069B0793FFF79CFF802313
:103260005B01C618802307001B039E4201D3F8268A
:10327000F60288235B05F31801931B68013302D023
:10328000019808F045FB3D49019808F051FB3B1DB2
:103290000293331D05938822029B52059B181B68DD
:1032A00008935A1C3CD044219AB20091402A04D879
:1032B0000320D11D814389B2009103991B0C8B42DD
:1032C00024D0402A22D80122300008A9FFF710FF9D
:1032D000021E1BD1380008A9FFF70AFF04000428CA
:1032E00031D9009A059B9B1880225201B218934253
:1032F00040D288235B05C118009A09A808F0D0FACB
:103300001D4B009A09A9F01808F072FA009A029B66
:103310009446634402931A4B029AFB189A42BAD31A
:1033200088235B05FC1821680198013908F000FB2F
:10333000200008F0EDFA039A07AB5A803000079995
:10334000FFF706FF0400002C03D1002079E70428D2
:10335000FBD988235B05E018069908F0E9FA0323F6
:10336000EA1C9A4300D16BE7034B0499E01808F07C
:103370003FFA65E70424ECE704000011FFFFFF7F3C
:10338000F80F0000F7B505001400402A21D80027E7
:1033900001AE71803780FFF7FEFE042816D93A008F
:1033A0003100FFF7A5FE042810D93688BC420BD0A7
:1033B000BD4209D0221CB44200D9321C064B92B245
:1033C000C118280008F06CFA30B2FEBDC04300B24C
:1033D000FBE703204042F8E70400001137B5042260
:1033E00004000D0001A81649FFF7CCFF02000428D5
:1033F0000BD1019BA34208D3AB4204D0104901A8D2
:103400000195FFF7F9FE01203EBD0E4C2368200018
:10341000019308F07DFA019920000139019108F02B
:1034200087FA80235B01E418074B9C42EED104220B
:10343000034901A80195FFF7DFFE0020E4E7C0463D
:103440005555000000C007110000081130B589B0C3
:1034500008F09EF910226946254808F061FA254BCC
:10346000009A9A420ED1019B029A0F2B33D8002169
:1034700001240698013B08D2002900D00292029B49
:10348000013331D10023029325E0551CF2D1020013
:103490002100EFE710341022200004A908F040FAC0
:1034A000029B013301D1069B0293882304995B059B
:1034B000C918059B06981A03120B049105928142C4
:1034C00003D02B4201D108F0EBF9019B013B0193A2
:1034D000019B002BDED1029B002B03D004930498A8
:1034E0004168084709B030BDE025014C2D03EFE7E6
:1034F00000000111504859368022F8B5964C974B80
:10350000D200002120001C6008F02AFB2300944A0E
:1035100088331A60934B1A786A23002A00D011333B
:10352000E3620A232365904B37221B780820A363AC
:103530008E4B2118E361102323628D4B3B25636181
:10354000C823DB00A36123008C331A602823013ACF
:10355000E26320646364CA67043A211DCA672100DC
:10356000BC310D602100C03108602100C4310B6006
:1035700021000635CC310D602100083DC8310D60B9
:103580002100D0310A602200D43210602200D832EB
:10359000136022000227E032210017604222DC3152
:1035A0000A6021001B3DE4310D602100E831086014
:1035B0002100EC310B6023000521F4331960230056
:1035C000F0331A602300183290331A6023009433CA
:1035D000186023001E3A98331A60AF23DB00236083
:1035E000644BFA262363644B644DE360644BF03113
:1035F000A3642300FF31FC33B600A16021611E608B
:10360000A5627325E5656D3D6565A56596255D4AF1
:10361000AD00E264666258606766A566002709250A
:10362000A767E566584F594D606720002567E26738
:103630003A6015279C30676007001A203860200028
:10364000A0300700212038602000A83007004C4837
:1036500038602000F830066026006427A436376002
:1036600026005F3FAC3637602600033FB036376038
:103670002600C637B436376026000027B8363760D4
:1036800038269E60424E96205E64424E5A66DE6147
:10369000414E9A645E62F53EFF3E9E621E269A6728
:1036A000354A8000DE661F675F67DD651D6618624C
:1036B000DA67BE23394A5B00E250394BD8382350D1
:1036C00004302250C4225200A350C623E4205B00E1
:1036D000E1500433334AE1503349344BD16034492B
:1036E000800019503349E938FF3819503249043005
:1036F000195032493248D16132491163324951631C
:103700001900F4310860CE20304940001160304982
:10371000195019002F48F83108602F49D1658221CE
:103720002E4A89005A501A002D490832D1671A00D2
:103730002C49B432116088212B4A89005A501A0052
:103740002A49883211602A4ADA6407F0B1FF012061
:1037500007F036FFF8BDC0460004FF1F4064FF1F9E
:10376000206FFF1F3044FF1F4A0AFF1F3A07000067
:1037700080C3C9019A020000DC0500006A1800003D
:1037800050C3000088130000F009FF1F204E000006
:103790006509FF1F68100000C409000040420F00C7
:1037A00010270000FC00FF1FC11BFF1F0000FF1FB0
:1037B000152CFF1FA52FFF1F3D2EFF1F811FFF1F71
:1037C0007126FF1F9D1FFF1F4921FF1F0D1FFF1F98
:1037D0009528FF1F7D29FF1FD918FF1FA127FF1F55
:1037E000C524FF1FD124FF1F0D1EFF1FC51EFF1F75
:1037F000851DFF1F0223F0B501245F4D5F4E2B7026
:103800005F4B91B01C705F4F039333680021200021
:10381000FB7006F0E9FD200006F0E0FC0023984272
:1038200005D0FA78552A02D0332A00D097E03360C9
:10383000042006F041FF07F00BFFFFF75DFE07F0E5
:103840003FFF1F22012400214F4B10AE1A704F4B37
:103850001C704F4B19704F4B19689143163A0A432D
:103860001A60602219689143403A0A431A6007F0CF
:103870003FFF07F085FFC120FF21474B80001A580A
:103880008A431A50C522920098588843BF39014391
:1038900099509858414908408021C901014380202E
:1038A00099509958C0050902090A0143995080218D
:1038B0003B48490108F0C4F8032322003949019428
:1038C0000093394808F06CF82C22384905A807F015
:1038D000E7FF05AC61782078023406F09FFCA64231
:1038E000F8D1334C334B226803201A40A023DB026B
:1038F00013432360802322689B04134323602268C0
:103900002D4B1A4080239B03134323602B4A2C4BDF
:10391000934200D8012007F063FF07F029FF8023BE
:103920002268DB0413432360287807F069FF039BB8
:103930001878C0B208F0F4F808F042F821490420E1
:1039400008F0E6F806F084FE00F0AAF800F0F8FDB2
:1039500000F0A0FE00F01AFA002011B0F0BD0093B4
:103960002100184A042008F04BF88023DB059C62F4
:10397000FFF76CFD5CE7C0464A0AFF1F34F00040C9
:103980003044FF1FCC61FF1F480AFF1F490AFF1F79
:10399000680AFF1FBCF0004000E100E0FF00FFFFED
:1039A0003444FF1FB856FF1F3454FF1F30BC0011B2
:1039B00014F00040FF7FF8FFFFFF9FFF0080FF1F14
:1039C000206FFF1F3B00010870B500252549264ADE
:1039D00026484D6308CA1B051B0DED188242F9D11C
:1039E00000268022224B92058B630921214B224C19
:1039F0001E62224B1120DA67214BDA688A43DA60B3
:103A00009A6820490A409A60266008F0C9F8112097
:103A100007F0E6FF636C1C4A13406364EE24E40085
:103A20006C431A4A200C0400642390420AD8FA22FC
:103A30003300D200904205D9154B0A21C01807F077
:103A4000FFFDC3B2134A11201372D48007F0E0FDCA
:103A5000114B1B78002B04D1104B1021187808F063
:103A6000A7F870BD00000540080605408006054027
:103A7000FF01000000F000400038004004E100E0D9
:103A80003CF00040FFDFFFFFFFFEFFFFB70B000031
:103A900030F8FFFFB461FF1FEE63FF1FEC61FF1FF3
:103AA000002210B51100112007F092FF10BD000098
:103AB000F8B500230926364F364C3B62E3681120E7
:103AC000B343E36007F08CFF112008F069F8112080
:103AD00008F016F840232268102513432360802342
:103AE0006268DB02134363608023A26802211343F0
:103AF000A360A368284A08201340A3608023A2681B
:103B00009B0113430122A360236CAB432364236C0A
:103B10001343236480231B013B62226B1F4B1A401B
:103B20002263626B1A406263A26B1A40A263E26B6B
:103B30001340E363E3681A4A1340E36006F06EFB48
:103B40000121082006F07EFC8023164A5B00516CA0
:103B500011200B43536407F03BFDFD21C720124B9E
:103B6000124A89005A50A36B80002B43A363E36879
:103B70000F4A3343E3600F4B195811408022120261
:103B80000A431A50802292051A600B4B5D63F8BD00
:103B900000F000403CF00040FFFFDFFFEFFFEFFFD1
:103BA000FFFF7FFF003800400000FF1FC9390011F0
:103BB000FF00FFFF00E100E00000054030B503A872
:103BC00004880B20002C0ED14968074D08784978ED
:103BD000090201430A20A94205D1012120001980D0
:103BE000024B1B7A137030BD192A0000B461FF1F0D
:103BF000F7B5150008AA16884A680F4F147852784E
:103C0000120222430A24BA4214D10122DBB20192E9
:103C100000962A0007F06CFC041E0BD1074B1B68B2
:103C2000002B07D068782A780002104342425041A6
:103C3000013098472000FEBD022900003861FF1FB7
:103C400030B5012503790400BFB02B4211D00A49D9
:103C5000408806F0B9FF28420BD0084B01A95B8DC4
:103C60004D800B80064B00221B7A60880B7104F09C
:103C70009DF83FB030BDC0463061FF1F6840FF1F58
:103C8000B461FF1F10B50549054806F053FF042134
:103C9000044A054806F010FF10BDC0463061FF1F02
:103CA000FFFF00005CBC00116840FF1F10B5024818
:103CB00004F0FEFE10BDC046413C0011012303701C
:103CC0000B4B1A7A4270022282709A78C270DA78AC
:103CD0000271032242711A7982715A79C2710C22DF
:103CE00002729A794272DB7983720B207047C04668
:103CF000B461FF1F022310B50370013B437005330D
:103D0000837010330371443B43712A33837144330E
:103D1000C37100230372064B04001B8843720A30F0
:103D2000FFF7CCFF831D0A30C0B2E37010BDC04660
:103D3000B461FF1F10B5142007F0CAFD124B142206
:103D40000021186007F00CFF002007F049FC01205B
:103D500007F036FF022007F01BFE032004F04CF9A9
:103D6000042006F061F9052003F08AFB062004F028
:103D700057F8072001F054FA082006F07DFE0920CC
:103D800001F03CF810BDC0463C61FF1F07F010FE7B
:103D9000012007F0CDFC07F033FF0000094B10B500
:103DA0000400984205D0012904D12000064906F0FC
:103DB000C1FE10BD0229FCD1013904F037FE0028F4
:103DC000F3D0F6E7FEFF00006261FF1F70B50D7AC9
:103DD000100004AA2C00168810221440154220D18D
:103DE000002E20D10A78022A18D14A685178157815
:103DF0000E4A09022943914205D00D4A914209D049
:103E00001C800A2404E014220A491A8007F048FDA5
:103E1000200070BD0C2208491A80F7E71C8001249D
:103E2000F6E70824F4E70B24F2E7C046F3FF0000AE
:103E3000F4FF0000BC42FF1F38BD001110B50400A4
:103E40000749084806F076FE074804F071FD002097
:103E5000E40704D50721054A054806F02DFE10BDEC
:103E60006261FF1FFFFF00009D3D0011A0BC00111B
:103E7000AC40FF1F00B50C4BBFB01A780B4902A82D
:103E800000F0C2FC6B4680B2D880002809D06A4698
:103E9000074B01A91B889380064B0022188803F06A
:103EA00085FF3FB000BDC0464061FF1F4161FF1F5D
:103EB0000641FF1F1042FF1F00B50C4BBFB01A7820
:103EC0000B4902A801F0B8FE6B4680B2D8800028EA
:103ED00009D06A46074B01A95B8D9380064B0022EF
:103EE000188803F063FF3FB000BDC0466A61FF1F42
:103EF0006B61FF1FAC40FF1F1042FF1FF7B50E00A4
:103F0000377A1C0008AB11003D001A8820231D40A1
:103F10001F423CD13378022B3BD173681F785B780A
:103F20001B023B431E4FBB4208D01E4FBB4214D066
:103F30001D4DAB4221D00A252800FEBD002A2AD102
:103F4000142C2AD82200F06807F0AAFC174B1C702A
:103F5000012CF1D9FFF7B0FFEEE7002A1BD1202C8E
:103F60001BD82200F06807F09BFC114B04211C7049
:103F7000104B187807F01CFEDEE7E3B20124009234
:103F800001940A00310007F0B3FA0500D4E70825D0
:103F9000D2E70125D0E70B25CEE70D25CCE7C046BB
:103FA000F3FF0000F4FF0000022900006A61FF1F18
:103FB0004061FF1FEC61FF1F332310B50400037045
:103FC0000A220749013007F06BFC064B0F201B68E3
:103FD0001A0AE37222731A0C1B0E6273A37310BDCC
:103FE000B461FF1FDC61FF1F30B5012503790400B8
:103FF000BFB02B4213D00B49408806F0E5FD2842A4
:104000000DD06A46084B02A81B889380FFF7D4FFA7
:104010006B46D8800022608801A903F0C7FE3FB03C
:1040200030BDC0466261FF1F0641FF1F10B5024848
:1040300004F03EFD10BDC046E93F001170B516000A
:1040400004AA148805AA15784A68507811780002E5
:104050002A4A0843801805284BD807F079FC031337
:104060001E29343F0720032C0BD80422121BAA421E
:1040700000D92A0022491A803000091907F010FCE3
:10408000002070BD0720112CFBD81222121BAA425F
:1040900000D92A001B491A80EEE707200E2CF0D821
:1040A0000F22121BAA4200D92A0017491A80E3E7FF
:1040B0000720032CE5D80422121BAA4200D92A00AB
:1040C00012491A80D8E70720032CDAD80422121BE1
:1040D000AA4200D92A000E491A80CDE70720032CF6
:1040E000CFD80422121BAA4200D92A0009491A80FB
:1040F000C2E700220A201A80C3E7C046DCD5FFFFD2
:10410000EBBC00118861FF1FDBBC0011D6BC0011A5
:10411000D1BC0011CCBC001110B50D21024A0348DE
:1041200006F0CAFC10BDC046C0BC00111C41FF1FF8
:10413000F0B50024274E85B03000B47100F0E2F8ED
:10414000254D264BEA89297C9A422FD10423300041
:1041500003AA00F057F90400300000F011F9012320
:10416000B371002C34D16B4699892B68C9BA4B4383
:1041700029891B4A1B145B1853806B46D9896B68CD
:1041800049BA89B24B4369891B0C5B181548191C45
:104190001BB2834200DD011C0B0400D500211388F3
:1041A000918001331380200005B0F0BD022722006A
:1041B00003AB3000009700F0F7F80E230400297CD1
:1041C0000122300000976B4400F0EEF80443C3E78F
:1041D0001C00E8E7F441FF1F9C61FF1F83050000FE
:1041E000B461FF1F0F27000073B5234E300000F0AD
:1041F00089F8224D07236A463000297C00F002F935
:1042000004003000002C33D16B461B787F2B2FD855
:1042100000F0B6F86B46D878F02302041B031A406E
:104220006B469B8816495BBA9BB21A432B68000900
:1042300053432A891B0C9B184B806B465A789B78FA
:1042400012031B011A436B68024353436A891B0C18
:104250009B180C481A1C1BB2834200DD021C13047D
:1042600000D500220B888A8001330B80200076BDA8
:1042700000F086F80124F9E7F441FF1F9C61FF1F5D
:10428000B461FF1F0F27000070B5114C237C002B79
:104290000FD0382B0ED10F4D280000F033F8CC236F
:1042A000AC222800217C9B0100F0F4F8280000F0EB
:1042B00067F870BD084BE2899A42FAD1054D280093
:1042C00000F020F800222800217C00F0C5F8EDE77E
:1042D0009C61FF1FF441FF1F8305000010B5084BD0
:1042E0001A7C002A09D05B69002B06D09847041E6F
:1042F00001D0FEF785FE200010BD0124F9E7C0467D
:104300009C61FF1F70B5C17905000C00631E9C41C4
:104310001A4BE402E41849000460C9B2007906F0BF
:10432000C7F8E979687949000131C9B206F0C0F8E7
:10433000E8790930C0B207F0E3FB0023E36661339C
:104340002360AA795B3B002A0ED022689A43023B85
:10435000134323600A23E3610733236200232363AB
:10436000A3630133E36370BD22689A4302231343BE
:104370002360462363610633A361EFE700500040EA
:1043800070B5002504000368DD66C0790930C0B24D
:1043900007F026FB2900207906F026F8290060792D
:1043A00006F022F870BD0000F8B51E0006AB1D78BF
:1043B000002304681700E366616007F0E9F9012350
:1043C0008022E3662B0027615200013B08D207F0F0
:1043D0007FFB08200A4A1168002D03D12800F8BD90
:1043E0002261F2E7236F034203D02369013D33705A
:1043F000013613685B1A032BEED90125EEE7C046A0
:104400006008FF1F70B51C00002305681600EB66EE
:10441000696007F0BDF901238022EB66230052009A
:10442000013B08D207F054FB08200A4A1168002C0F
:1044300003D1200070BD2A61F2E72B6F034203D045
:104440002B69013C3370013613685B1A032BEED9DC
:104450000124EEE76008FF1F002370B50468150013
:10446000E366616007F094F90123E366256107F0D4
:104470002FFB8020064A80001168636B034205D140
:1044800013685B1A032BF8D9012070BD0020FCE7EC
:104490006008FF1F70B51D00002304681600E36666
:1044A000616007F075F90123E36626610F33626BE3
:1044B0001A42FCD02B0A23611023626B1A42FCD0F3
:1044C000EDB2256107F004FB8020074A80001168E7
:1044D000636B034205D113685B1A032BF8D90120E3
:1044E00070BD0020FCE7C0466008FF1F70B51E00CD
:1044F000002305681400EB66696007F049F90123A1
:10450000A619EB660F33B4420ED107F0E1FA802012
:104510000A4A800011686B6B03420CD113685B1A66
:10452000032BF8D9012070BD21782961696B1942EC
:10453000FCD00134E7E70020F5E7C0466008FF1F24
:1045400010B5084CE368002B08D18022064B5202BC
:104550001B689B186360054B1B68236007F018FB02
:10456000A06010BDDC61FF1FC8F00040CCF000402F
:1045700070B5184A936A916A9942FBD116498A68C4
:104580009A421FD39A1A8B60144B0126186893B273
:10459000D202D20E4343424300204C681B0A1B192F
:1045A00012029B180E4C0A684B60551CA3420CD893
:1045B000002801D04B600A600A4A136008680A4B61
:1045C000186070BD581E821ADDE7084A30009B183B
:1045D0002A00EAE700F00040DC61FF1F140AFF1F19
:1045E00040420F00C8F00040CCF00040C0BDF0FFDA
:1045F00070B51F4C23793F2B01D93F2323711D4BED
:1046000022791A701878C0B207F072FA18231A4982
:104610001A4A0B801A4913800B805380A3791949D9
:1046200080200B800C21938001334B43164D191CC5
:104630000001834200D9011C2980D1806379002BBD
:1046400011D101336371237A012B01D80223237224
:104650006279237A0D4853430A21584306F0F0FF4C
:104660000B4D286070BDA02BEDD9A023EAE7C04612
:10467000D061FF1F480AFF1F0E42FF1FDC43FF1FD0
:104680000C42FF1F0A42FF1F0842FF1F7102000079
:10469000C061FF1FF8B515210020FEF79FFE114CE9
:1046A000011E114D09D10C22104BC1CBC1C42800F1
:1046B00007F056FAFFF79CFFF8BD0C2220000C49CA
:1046C000FEF760FE0C2802D0084B43CB43C40C22FB
:1046D00028000849FEF756FE0C28EBD00C220021DA
:1046E000E5E7C046D061FF1F9C61FF1F2CBD001194
:1046F000FC0C0000F50C0000F0B51D4C8022A54418
:104700000400882069465201400507F0A1F8902274
:1047100012016A441300200032C832C316C816C3FF
:104720008023144C144FA6689B033343A3603B6063
:1047300007F0BEF98823A0685B05C01807F0E8F809
:104740000025882329008022A0685B05C018401935
:104750006944520007F04CF880230135FF355B01B6
:104760009D42EED1A6603E60044B9D44F0BDC04624
:10477000FCEFFFFF4C43FF1F9808FF1F04100000D1
:10478000F0B5040087B0002825D0684606F0E8FFA1
:104790001B4C022806D106226946200007F078F952
:1047A000002816D06946002301250F262F00E25C61
:1047B000013310091030874038002F0032409740F5
:1047C0003A0002434A610439062BEFD16846FFF7ED
:1047D00093FF07B0F0BD182269460A4807F038F881
:1047E0006A46A300D358013305D01822FF2168463A
:1047F00007F0B6F9EAE70134062CF1D1E9E7C04643
:104800006509FF1F00090011F0B5002504000E0026
:1048100085B0AA4200D186E04B1C087801934B7802
:104820008978377909021943F3783F061B040B4353
:104830001F43039720706570252800D196E033D878
:10484000112813D806F0E4FF69002B012B012B017E
:104850002B01AA00B800B1002B012B012B012B0169
:104860002B012B012B012B0105012501232800D150
:10487000DEE0DB2800D034E1042A00D8ACE01025CB
:10488000052A05D0551F2A003800711D07F008F8C9
:1048900005223100200007F003F82A003900601DCE
:1048A00006F0FEFF05353EE0562859D010D83328D3
:1048B00000D19DE0552839D02628DAD19F4B290018
:1048C000132218001D0007F04BF9FEF799FB5CE07E
:1048D000712800D177E0722800D180E0602800D1F3
:1048E0008BE0DC28C5D1022A00D875E07378BFB20E
:1048F0006370B378A370032A05D0033A390092B2EB
:10490000F01CFEF779FC10223900E01CFEF73AFD9E
:10491000C51C002807DA60705CE00C222000884982
:1049200006F0BEFF0C25280005B0F0BD013A854D0C
:104930000C2A13D8002A0AD02800019906F0B0FFEB
:10494000FFF756FE0C2228007F49FEF755FC290090
:104950000C22601C06F0A4FF0D25E4E70C22EBE717
:10496000784D7A4B2A0043CB43C2E9E7013A734DB5
:104970000C2A11D8002A08D00199280006F090FFCF
:104980000C2228007249FEF737FC29001322601C14
:1049900006F086FF1425C6E70C22EDE705226D49D7
:1049A000601C06F07DFF0625BDE712226A49601CE7
:1049B00006F076FF1325B6E708226849601C06F06A
:1049C0006FFF0925AFE77178F02905D8644B188887
:1049D00001F08EFD0225A6E7FF236370FAE7614B25
:1049E000012A03D072789A706270F3E79B78F4E73B
:1049F0002000FFF7E1FA050095E7013A594B5A4DBF
:104A0000072A10D8002A10D00121280059700199D6
:104A100006F046FF01F04AF829000722601C06F064
:104A20003FFF08257FE70722EEE700225A70F3E7F1
:104A3000042A04D94D4D2F6007F0AAF8A860FFF7AB
:104A400097FD0422039003A9601C06F029FF0525A9
:104A500069E7474D062A15D906222800019907F073
:104A600017F800280ED006220199280006F018FF3A
:104A7000062240492800FEF7BFFB0123394A9178FE
:104A80000B43937029000622601C06F009FF0725DE
:104A900049E7012AA0D07078FFF772FE9AE7012853
:104AA00000D0E6E6931E344F132B04D87378002B06
:104AB00009D100F015F9314B39001D78601C6A1ED0
:104AC00006F0EEFE2FE7551E2A000199380006F089
:104AD000E7FE2B49AAB23800FEF78EFB00F038F94A
:104AE000E9E7DA281DD1042A00D875E7082A15D984
:104AF000B37972791B021343F27912041A43337AA1
:104B00001B0613433B603B680522310020000393E2
:104B100006F0C6FE0422601D03A950E7FE23637061
:104B2000F1E7DE2800D057E7511E012A01D1002508
:104B3000F9E6019800F0A0FFF9E7C0469C61FF1F6D
:104B400038BD0011D061FF1FFC0C00002CBD00110E
:104B5000F50C0000A861FF1F8861FF1F5043FF1F75
:104B60001042FF1FCC61FF1FAD42FF1FDC61FF1F22
:104B70006509FF1FADAC0000CD63FF1FCB63FF1FB6
:104B8000AEDE000070477047020010B5094B0A32D4
:104B9000094C92B2DA815A8298811882207802F008
:104BA0000DFB0422054B012120781A7007F000F854
:104BB00010BDC046DA42FF1F1664FF1F1564FF1FB9
:104BC000013870B5042809D806F0C2FE0309280888
:104BD0001200234B0221187806F0EAFF70BD204B2B
:104BE0000821187806F01CFE00221E4B1A72F5E709
:104BF000802200241B4B1A4D52001A8108211A688A
:104C00002878DC7206F01CFE2100287807F000F8F6
:104C1000012000F051FE00F049FFDFE7104B0821B2
:104C2000187806F0FDFD1048FFF764F80F4B104AA6
:104C30009B79002093800F4A13808022094B5200F9
:104C4000D8721A8100F038FE00F030FF0A4B9B78D2
:104C5000002BC3D0094A136006F072FEBEE7C046BF
:104C6000EC61FF1FC061FF1F1942FF1FD061FF1FD2
:104C7000DC43FF1F0A42FF1FCC61FF1F34F00040DE
:104C800010B501290BD1012809D1054B1B78002B48
:104C900005D02622034B04485A72FFF775FF10BD5A
:104CA000EE63FF1FC061FF1FC40900000300F0B5E1
:104CB0000A4D8E18B14202D152008018F0BD0C7816
:104CC0002F6824093C5D0F271C700C7801313C4093
:104CD0002F683C5D5C700233ECE7C0460442FF1F66
:104CE0000D22124B10B51A700C23114C1149237070
:104CF000093A033B1048637006F0D2FD2D230122D0
:104D00000E490F48A371FFF7D1FF01220D49FFF7AC
:104D1000CDFF01220C49FFF7C9FF030000200B491A
:104D200002001870FEF768FA10BDC046EA63FF1F64
:104D3000CB63FF1FEBBC0011CD63FF1F6709FF1F93
:104D4000D263FF1F6609FF1F6509FF1FAEDE00006B
:104D500070B5124C142220001149FEF713FB431EBC
:104D6000104D132B17D8AB78002B14D0431C2B708D
:104D700009236B7000230019037028782900013083
:104D8000C0B206F0ADFC297822000139C9B200207A
:104D900005F0B0FD70BDFFF7A3FFEEE7CD63FF1F89
:104DA000AEDE0000CB63FF1F10B5114B1A781870F0
:104DB000002A0ED000280BD10E4B1A78062A07D8ED
:104DC0005423D340DB0703D50B4B187802F0F6F9D8
:104DD00010BD0028FCD0074B1B78012B02D0033BF1
:104DE000022BF5D8044B0121187806F0E1FEEFE71D
:104DF000EE63FF1F1564FF1F1664FF1F70B54A4E58
:104E00004A4A4B493070012005F000FC00F0B2FE28
:104E1000FEF7F6F806F0B4FD032246494648FFF7D0
:104E200045FF2D24030004221C7044490130FFF784
:104E30003DFF30230470424D424C437083702E3B43
:104E4000062220004049EB87FEF79CFA062813D083
:104E5000200006F085FC022809D00321200006F07E
:104E600037FC8D23E3706E3B237119336371062287
:104E700020003549FEF7C0F9344B1B68FC335C64F5
:104E8000FFF766FF0020FFF78FFF314C314A012109
:104E9000314B1278207802F053F9304A304B1278B7
:104EA0000021207802F04CF901222E4B1A702E4B73
:104EB000DB78552B31D12D4B3B325A722C4B2D4A7E
:104EC000AB81EA812B826A822021307806F0D8FB00
:104ED0000120404205F05AFD0120404205F0F6FD58
:104EE000FFF71AF9FEF7CEFE00F0A4FC01204042C5
:104EF000FEF7A4FF012006F0BBFDF02001F0DCFA74
:104F00000121307806F054FE307802F0B3FA1A48E6
:104F100006F0A6FCFEF7CCFD70BD6422174B5B7952
:104F200053431A000A32CBE7EC61FF1F854B001197
:104F3000814C00115043FF1F8861FF1FA861FF1FB4
:104F4000DA42FF1F6509FF1FADAC00004064FF1F80
:104F50001664FF1F3842FF1F1942FF1FEA63FF1F3D
:104F6000CB63FF1FBC63FF1FCC61FF1FC061FF1F2E
:104F7000C4090000CE090000EE61FF1FD061FF1FD1
:104F8000F8B50A0020230D001A40194257D0574B9C
:104F90001B78002B50D0FFF7EBFA554B554C564E73
:104FA00099686268737A8A1ADB039A4202D3616055
:104FB000FEF77EFD327A217A531EDBB2994205D18B
:104FC000FFF762F9002000F0A7FD0FE09142F9D34E
:104FD00000232372FFF782F9012000F09DFD474F67
:104FE0003800FEF787FE390006F022FD637A002BB9
:104FF0001FD0013BDBB26372002B1AD1404BDB7830
:10500000552B01D106F09CFCE37A002B0CD0002339
:105010003C4A3A4FE3721388380001331380FEF79D
:1050200069FE390006F004FD642370795843FFF7E8
:10503000ABFD237A0133237220206840F8BD0BB208
:10504000002B0ADA304B187806F05AFB002801D002
:1050500006F096FD80200002EFE70224214206D0F0
:10506000244B01201A72FFF79FFE2000E5E70B0793
:105070001ED5FFF77DFA1E4B1E491F4C98684A68E3
:10508000637A821ADB039A4202D34860FEF710FD6E
:10509000FFF724F9FFF7F8F8012000F03DFD00F0DC
:1050A000E3FB2368DB0701D5FEF7C0FF0820C4E758
:1050B0001024214206D00D4B1B78002BD5D1FEF7D2
:1050C000F5FDD2E70124214207D0104800F06CF82A
:1050D00006F0DEFB00F006FDC7E7042408002040D0
:1050E0002142ABD0FEF7C6FEBFE7C046EE63FF1F0E
:1050F000DC61FF1FC061FF1FD061FF1F1942FF1F4E
:10510000CC61FF1FB461FF1FEC61FF1FFC41FF1F5B
:10511000F0B51B4B1B4F1B883A8804001A4E1B4DE1
:1051200085B09A420DD832889A420AD3184B1A8811
:105130002B889A4205D1174A174B12881B889A422E
:105140001BD0052001F00EFA3B8802AA1380338899
:10515000019053802B88114D93800F4B02A91B881F
:10516000D3800F4B2A78188802F02AFF0D4B0821B4
:105170002878019A1C7006F0D3FA05B0F0BDC0463D
:10518000BA63FF1F0E42FF1F0C42FF1F0A42FF1FA0
:10519000B863FF1FB663FF1F0842FF1F1664FF1F9F
:1051A0001042FF1FB463FF1F13B50C4B1C78002C7B
:1051B00011D1002801D00A4B18600A4A0A4B117815
:1051C0000A4A10780A4A01920A4A0092002205F01F
:1051D00089FA200016BD1124FBE7C0461564FF1FA5
:1051E000B063FF1F1464FF1F0464FF1F1664FF1FDA
:1051F000F063FF1FF463FF1F10B5064B12201B78EE
:10520000052B06D1044B13221988044B187801F0A2
:1052100085FB10BD1564FF1F1042FF1F1664FF1FA2
:1052200010B500240122114B52421870104B1C7013
:10523000104B1A8002F01EF904220F4B21001A7045
:105240000E480C3206F074FC102221000C4806F0C7
:105250006FFC07220B4B1C600B4B1C700B4B1C7024
:105260000B4B1A700B4B1C7010BDC0461664FF1F11
:105270001564FF1F1042FF1F1464FF1F0464FF1F0B
:10528000F463FF1FF063FF1FCA63FF1FC963FF1FA3
:105290001242FF1FC863FF1FF8B5174C06002578A0
:1052A00006A814240078052D23D1B41F134FA5B2EE
:1052B0001824BD421DD88D1FADB2BD4219D8FA25A4
:1052C0006D00AA4215D21D000D4F0A3DADB2BD4280
:1052D0000FD80C4C26800C4C21800C4900240A80ED
:1052E0000B4A1380FFF714FF0A4B0421187806F0CD
:1052F00097FA2000F8BDC0461564FF1F790C000026
:10530000750C00000E42FF1F0C42FF1F0A42FF1FD8
:105310000842FF1F1664FF1FF0B50BB20D0089B0E5
:10532000002B00DB70E1A44E307806F0E9F9041E92
:1053300050D00378A22B00D122E1D02B1AD0912B90
:1053400045D143780E2B42D19C4B82889A423ED164
:105350009B4A83681278052A39D1032018567F2882
:1053600035D0984B1B68002B31D05B68002B2ED0BA
:1053700098472CE08078072829D806F0E9FA042815
:10538000183F3F74A8D86378002B0CD101218C4BB7
:1053900019708D4B1A78002A5BD08C4B307801F055
:1053A000CFFE002855D00722854B1A7051E0617856
:1053B0000029F8D1E378002B11D0854A854B12786B
:1053C000307801F0BDFE60706378002BEBD12000D7
:1053D00006F0D6FB80200002684009B0F0BD784B93
:1053E0001B78022BF3D00121307806F059FB0028FE
:1053F000EAD10121307806F0DBFBE5E76378002B8A
:10540000D1D16F4F032807D13B78052B02D101334F
:105410003B701EE00223FBE76F4B1A886F4B029331
:10542000002A0BD01B78002B03D00121307806F026
:1054300077F93B78062B04D1013BE9E7029B1A7010
:10544000F7E7042B41D10121029B3078197006F057
:10545000AFFB5C4B1B68002BB9D01B68002BB6D090
:10546000574A107884E76378554F002B27D10622DE
:10547000211D5B4806F014FA62895A4B5A491A807A
:10548000A2895A4B1A80E3890B800521397058494B
:105490000A80584A1380228A574B1A80574B1B7830
:1054A000012B09D11F2001F05DF8FA22920042433E
:1054B0000421307806F034F90022484B75E7312B8F
:1054C00000D070E70022454B1A700323A0E70622A4
:1054D0000021434806F02CFB0023454A0421138099
:1054E000444A30781380444A138006F099F9082121
:1054F000307806F095F9A379083B5A425341304A77
:1055000003331370304B1B78002B06D0334B3078AD
:105510001A78002A06D001F051FE0122314B524286
:105520001A8096E70121197006F042FBF5E7082181
:10553000307806F075F96378002B00D047E72C4BE4
:105540002D4F0293E388029A04211380294B30786F
:1055500003932389039A138063893B8006F0A0FAA2
:10556000002800D033E7264B1B68002B00D12EE724
:10557000039902983A88098800881B68984726E7AB
:105580004379132B00D022E70389012B0AD11D4B4D
:105590001B78022B06D10821307806F041F9FFF77D
:1055A0002BFE14E7052000F0DDFF08210200307813
:1055B00006F0B6F80BE7C0461664FF1F051400009E
:1055C0001564FF1FB063FF1F3842FF1F1942FF1F02
:1055D000EA63FF1FCB63FF1FEC63FF1FEE63FF1F38
:1055E000BD63FF1F1042FF1FC463FF1FC663FF1F81
:1055F000BA63FF1FB863FF1FB663FF1FBC63FF1FC3
:10560000AC63FF1FB463FF1F8020C001014200D0C4
:10561000E2E6CB0731D5324B1B78002B1DD0314E43
:1056200005AC3378052B1AD1023B23702E4B210099
:105630001B7823722D4B1B7863722D4B187801F069
:1056400023FD002809D007202A4B30701B68002B4F
:1056500003D01B68002B00D098470120BCE60E2029
:10566000254B06221B7825492370254B1B78637038
:1056700002ABC01806F014F9D8E70223080018405E
:10568000194209D0174B1B78052B03D11D4B1888E5
:1056900006F0BEF902209FE60424214203D0FFF762
:1056A00037FD200098E6082308001840194200D171
:1056B00093E6154B1C78012C03D0022C0DD008204A
:1056C0008AE6124B124A134913481B88128809882C
:1056D00000880094FFF7E0FDF1E7FFF78DFDEEE7AE
:1056E000EE63FF1F1564FF1F1242FF1FC863FF1FF9
:1056F0001664FF1FB063FF1FCA63FF1F1342FF1F23
:10570000C963FF1F1042FF1FB463FF1F0842FF1F42
:105710000A42FF1F0C42FF1F0E42FF1F10B502A8D6
:1057200004880B20002C10D14968087849780902B8
:1057300001430C48814209D1022119800A4B598842
:105740001170DB7800205BB2537010BD074C0A204B
:10575000A142FAD102211980034B998811705B791B
:10576000F0E7C0466E2A0000B461FF1F6F2A0000F8
:10577000F7B5150008AA16884A680F4F14785278B2
:10578000120222430A24BA4214D10122DBB201924E
:1057900000962A0005F0ACFE041E0BD1074B1B68D7
:1057A000002B07D068782A7800021043424250410B
:1057B000013098472000FEBD022900002864FF1F29
:1057C00030B5012503790400BFB02B4225D0144920
:1057D000408805F0F9F928420CD0124B01A95B8DE5
:1057E00000220B8002234B800F4B5B888B806088EC
:1057F00002F0DCFA0D49608805F0E6F9C0070CD527
:105800000B4B01A91B8800220B8002234B80064B07
:105810009B888B80608802F0C9FA3FB030BDC046DB
:105820002064FF1F3C42FF1FB461FF1F1864FF1F6D
:105830009642FF1F10B5074C0749200005F07AF982
:105840002000064905F076F90721054A054805F0CC
:1058500033F910BDFFFF00002064FF1F1864FF1F15
:1058600058BD00113C42FF1F10B5024803F020F95B
:1058700010BDC046C15700110221430888400B40AB
:105880000A31084003430E20024AD17881430B437A
:10589000D3707047AD42FF1F064A1379410705D503
:1058A00080210B4380011371907170477F210B4061
:1058B000F8E7C046AD42FF1F054A5378002803D0E1
:1058C00080210B43537070477F210B40FAE7C0469D
:1058D000AD42FF1F0F21114BDA780A40DA705028D1
:1058E00010D901310A43DA702022D9780A43DA70DC
:1058F0004022D9780A43DA708022D97852420A438A
:10590000DA7005E03C28EFD82828F1D81428F3D81D
:105910000122D9780A43DA707047C046AD42FF1FB2
:10592000F8B57F23324D04006E789E43314B984288
:1059300005DD76232B70363B33436B70F8BD2E4B61
:10594000984203DA58232B701433F5E783B21A0018
:1059500000215F32294892B2294F297082422DD905
:10596000A9708C4203DA5B421CB220232B700534F1
:1059700020B20A2105F064FE04B2FA239B009C4287
:1059800033DB80232A785B4213432B706421200091
:1059900005F056FE0A2100B205F0E2FF09B22A78AE
:1059A0007B5C13432B700A21200005F049FE0A217D
:1059B00000B205F0D5FF09B27B5C0AE08022AA7034
:1059C000002CDADA5B421CB220232B705F23092CF7
:1059D000E9DC1E430A2120006E7005F0C1FF09B208
:1059E000AA787B5C1343AB70A8E7632CCEDCEDE7B1
:1059F000AD42FF1F1B4E00001DFCFFFF2A080000E8
:105A000082BD00117F23F7B5194FCD013E79040007
:105A10009E433E71EDB2632806DD093B33433B7183
:105A200040231D437D71F7BD0300093304DA582379
:105A300033433B716C23F4E70E4B019300280BDAE0
:105A40000423444224B23B710A21200005F088FF60
:105A5000019B09B25B5CE4E70928F5DD0A2105F04A
:105A6000EFFD019B00B21B5C1E433E71ECE7C0469C
:105A7000AD42FF1F82BD0011F8B50A4F05003B780B
:105A80000E00002B0CD0084C2000FEF73BFC33002E
:105A90002A0020003978FEF729FD2000FEF770FC6F
:105AA000F8BDC0463464FF1FB442FF1F70B50A4EF4
:105AB0000A4D07223100280005F0EAFF002809D02E
:105AC000074C31000722280005F0EAFE08212000DB
:105AD000FFF7D2FF70BDC046AD42FF1F2D64FF1F10
:105AE0002C64FF1F7F2210B50A4B59789143033A6B
:105AF0001A70103A0A435A7078220E219A70DA7896
:105B00008A43DA7006221A7137325A71FFF7CEFFD4
:105B100010BDC046AD42FF1F10B5002824D0134C65
:105B20000A210223E05E05F08BFD00B2FFF7F8FECC
:105B30000423E05E642105F083FD012100B2FFF73C
:105B400061FF207AFFF7C6FE0320FFF795FE0020D5
:105B5000FFF7A2FE064B1878053843425841C0B201
:105B6000FFF7AAFEFFF7A2FF10BDC046B461FF1FFA
:105B70001564FF1F70B50024094D2800AC71FEF7B5
:105B8000C1FB10233E212800064AFEF7AFFCA042CD
:105B900000D13E34044B28001C70FEF7F1FB70BDB1
:105BA000B442FF1F72BD00113464FF1F0200F0B544
:105BB00001270A480A4E51188B1A002B00DCF0BD51
:105BC000082415784308684038404000805B013C59
:105BD00058406D08002CF5D10132EDE7FFFF0000C1
:105BE00092BD0011F0B500250F269D4200DBF0BDEF
:105BF0004C5D070944403440A400A058013578406A
:105C0000F3E70000F0B589B06A460D000B000F27DE
:105C1000110010351C780133260024093E4016700F
:105C200054700232AB42F5D12023024AFFF7DAFF6B
:105C300009B0F0BD98BD0011F0B54E780B7889B071
:105C400036020C00170001901E43012A61D9954BC2
:105C50009E4200D877E001339E421CD1062A17D11C
:105C6000CA788B7812021A430B791B0413434A79C2
:105C700012061A438C4B5A6100221A705A808B4AC2
:105C80005A608B4A9A608B4ADA60002009B0F0BDF6
:105C900088225205EEE7884B9E423CD182498B78A0
:105CA000002B00D0F6E00C2A31D10F22A3789343C9
:105CB000E278120213432279120413436279120626
:105CC00013434B60E279A07912020243207A000468
:105CD0001043627A12060243CA60E27AA07A120284
:105CE000024376484A81834208D804236E4914222D
:105CF00001980B7005F0D4FD1420C7E71201D218EB
:105D000089235B059A42F0D801238B70BDE7022AF4
:105D1000FAD00523EAE76A4A01239642E6D1FFF763
:105D20006BFA052F0CD9E378A2781B021343227972
:105D300012041A4363791B061343624A03931360E8
:105D400005F0FEFDA1E7584D2B78002B9DD1AB78D7
:105D5000002B00D1A0E02B8901339BB20093B3420A
:105D600000D091E0132AD4D9CF7C8B7C3F02122142
:105D700020001F43FFF71AFF874200D08EE0002E5D
:105D80003DD1E378A2781B0213432279E96812041B
:105D90001A4363791B06134303930A228B4212D1E1
:105DA000FF23A370E370237163716B89002B09D10A
:105DB000E37B227C1B0212041343A27B13431B09C7
:105DC00001336B8100226B89002B8ED0002A67D1B2
:105DD000686837013818000B6B690003039098421C
:105DE00005D9686105F094FDEB780133EB706868C4
:105DF0001022A11C381805F0FBFC2E8145E76F89A5
:105E0000009A7B1E9BB293423AD1E278A3781202A9
:105E10001A43237905A81B04134362796C681206A0
:105E20001A43EB6800920392211D0C22049305F0A3
:105E300037FD0120260004A940421036FFF7E2FE9C
:105E4000013F012F17D1009A0B232861824200D015
:105E50004CE704221C49200005F0CAFC042203A9D7
:105E6000686805F0F5FCE968039AFF23914200D1C8
:105E70003CE7F73B3AE73100FFF7C4FE1036DFE7B7
:105E80000923B742A4D831E7009BB34200D9FCE60E
:105E900007232BE7022329E7032327E7062325E728
:105EA0000A2323E7FFFE0000BC42FF1F0000011190
:105EB000FFFF00005048593601FF0000FFFF0011AE
:105EC00002FF000034F00040C842FF1F10B5034C31
:105ED0000B000122210000F06BFA10BD8D60001153
:105EE0000B8870B506000D000224162B11D92B006B
:105EF0000322094900F05CFA041E0AD1074B2A88E4
:105F00001B88191C934200D9111C300089B200F083
:105F1000EFFA200070BDC046B96000115A64FF1F3F
:105F200010B54A780400013A0B000220012A07D874
:105F30000A78002A04D005222000024900F038FA2D
:105F400010BDC046E76000110A7810B50B000400D0
:105F50000220002A04D007222000024900F028FA7B
:105F600010BDC046936100110A7810B50B00040003
:105F70000220002A04D009222000024900F018FA69
:105F800010BDC046F961001110B5034C0B000B2287
:105F9000210000F00DFA10BD2962001110B5034C6C
:105FA0000B000D22210000F003FA10BD9B620011CE
:105FB00010B5034C0B000F22210000F0F9F910BDC1
:105FC000F56200110A7810B50B0004000220002AC7
:105FD00004D011222000024900F0EAF910BDC046A9
:105FE00005630011002310B51322190000F0E0F939
:105FF00010BD000010B5034C0B001722210000F06B
:10600000D7F910BD57630011002310B519221900EC
:1060100000F0CEF910BD000010B5034C0B001B22A0
:10602000210000F0C5F910BD91630011F7B5848916
:106030000D0006000121002C22D000238268D356D7
:106040001778002B1EDA0C2C1AD90C3CA4B21319A9
:1060500040880093230002F086FE431E98410130E1
:106060007B06DB0F6B703F23013C1F40A4B22870FE
:10607000AF70AC80002C07D0B3680133AB60002157
:106080000800FEBD0020EBE7AC60F8E70B7803707A
:106090004B8843704B881B0A83700B79C3700420B4
:1060A00070470420022B06D10020537811781B0280
:1060B000009A0B43138070470B8803700B881B0AF0
:1060C0004370022070470420009983420AD153781C
:1060D00010781B0203430B80D37890781B02034394
:1060E00000204B807047F8B50D004B78012400214B
:1060F000461C03702B788B4201D82000F8BD6B78CA
:10610000B01C4F1C012B10D1890069184B8802224A
:1061100033704B88B9001B0A7370691805F068FC6E
:1061200004360434A4B2F9B2E4E7122359436B18DD
:106130005A88043132705B8810221B0A7370691808
:1061400005F056FC12361234ECE770B5049D1400CD
:106150001E00052B01D8042070BD637812781B0245
:1061600013432B80E378A2781B02134302226B8037
:106170002A71211D681D063E05F03AFCB2B22A8143
:10618000E92AE8D82800A11D0A3005F031FC0020DA
:10619000E2E7002310B50A789A4201D8900010BDBA
:1061A0009A008A185488013304705488DBB2240A98
:1061B0004470948884709288120AC2700430EAE7AE
:1061C00010B51100029C062B04D004201022142BC1
:1061D00001D010BD022222714B7808781B020343C4
:1061E0002380CB7888781B02034363800431601DD1
:1061F00005F0FEFB0020ECE710B50C788B7804313D
:106200005C43E4B203702200013005F0F1FB601C36
:1062100010BD0420022B06D10020537811781B02F8
:10622000009A0B431380704710B50C000A880231A6
:1062300005F0DEFB208810BD70B504000D00049849
:106240001100012B01D8042070BD1678527812027B
:10625000324302800200F13255701470E125002CA7
:1062600000D10C35023B9AB24280AA42EBD80231EF
:10627000043005F0BDFB0020E6E7042000998342CE
:106280000AD1537810781B0203430B80D37890789F
:106290001B02034300204B80704710B50C000A8896
:1062A000023105F0A5FB208810BD000070B501216A
:1062B0001E000420049C0E400B4218D1CB40DDB2DE
:1062C0008D4214D90A49DBB2098899420FD32300C1
:1062D000EE331D703300580011184978165C09021E
:1062E000314301332152D9B28D42F4D8002070BD20
:1062F000D442FF1F10B50C000A88023105F078FB6C
:10630000208810BD10B50C788B7804315C43E4B262
:1063100003702200013005F06BFB601C10BD10B54E
:1063200011000298032B01D8042010BD1478527874
:10633000043B120222430280CA788C781202224364
:1063400042809AB28280EB2AEED80431063005F002
:106350004FFB0020E9E710B50C000B8803700B8899
:106360001B0A43704B8883704B881B0AC3708A8852
:106370000430063105F03CFBA088043080B210BD2B
:106380000420012B03D100201378009A137070476A
:1063900010B50C000B8803700B881B0A43704A88E9
:1063A0000230043105F024FB6088023080B210BD59
:1063B000F0B589B003931E4B029242000700D05AF9
:1063C000019102F020F81325061E2DD0029B012416
:1063D0000370019B002B04D0001903999847001902
:1063E00084B26B461B7A5BB2002B0FDA10213800A7
:1063F00002F01CFB1925002813D130003219E1B23C
:1064000002F066FC051E0CD10C34A4B2042304AACD
:10641000380005A993800696948101F0AFFD051E12
:1064200002D0300005F024FA280009B0F0BDC046C3
:106430005864FF1F70B505000C0000280CD0002028
:10644000814209D010222000044905F0D1FA012030
:106450002B7823736B78637370BDC046D8BD001171
:10646000F0B506000D0017001C0085B002291BD0F6
:106470000020102907D1022B07D0102B03D115E0E3
:106480000020102C08D005B0F0BD69463800FFF799
:10649000D1FF2A0069460BE069463000FFF7CAFFCA
:1064A00022006946380004E0022BE9D12A003900B5
:1064B000300005F05DFAE6E7031CF02800D9F02370
:1064C000032008499AB2013A0B80D31703400649CA
:1064D0009B189B100B80D30F04499B185B100B80FB
:1064E0007047C046D842FF1FD642FF1FD442FF1F4D
:1064F000034B1B888B4202D3024B4000C1527047B2
:10650000D842FF1F5864FF1F014B4000185A7047C4
:106510005864FF1F1722014B1A8070475864FF1FF1
:1065200070B505000E2005F0ABF9041E13D0D02382
:10653000037000230622837007494570033005F07D
:1065400057FA064B2100DA8A62811B7E2373044BC3
:10655000187805F055F870BD7464FF1F6464FF1F60
:106560002843FF1F262803D8024B4000C05A70471B
:106570000148FCE7DA42FF1FFFFF000070B506008C
:106580000C00094D1C220021280005F0D1FA074B10
:106590001E70074B1C7005F023FB0123002801D05F
:1065A000002312202B7070BD6464FF1F2843FF1F5F
:1065B0008564FF1F70B505000D4C0800E260A16006
:1065C00010220021656005F02BFA012803D110216B
:1065D000A06802F058FD10220021280005F020FAE2
:1065E000012803D11021606802F04DFD70BDC04646
:1065F0006464FF1F70B5041E05D1002903D0062274
:106600000D4805F0F5F90D4B1D78012D11D1002C29
:1066100005D102221A7005F04BF9280070BD002246
:106620001A70074B1B78FF2BF7D02000FFF778FF7D
:10663000F3E70025F1E7C0467464FF1F6464FF1FA1
:106640002843FF1F030010B5002801D1002010BD12
:1066500000780B4A002803D15988D1821B79137620
:106660001378022BF2D10023984200D10333137028
:10667000044B1B78FF2B01D0FFF752FF0120E6E708
:106680006464FF1F2843FF1F002911D000280CD08D
:106690004B79012803D140225242134303E03F22A9
:1066A0001340032802D001204B7170474022F4E7C9
:1066B0000800FAE770B5094D0100287800280BD0D2
:1066C000074C0622200005F093F921002878FFF7F7
:1066D000DBFF200005F0D4F970BDC0468464FF1FC5
:1066E0005E64FF1F00290AD0012808D13F224B79A0
:1066F0009343C02B03D0403B5A425341981C7047F0
:1067000070B5174D06002B78FF2B15D00A2005F029
:10671000B7F8041E10D0D0230370C83B8370114B10
:1067200011491B784670C3700622043005F060F9E9
:106730002100287804F064FF0C4B1B78012B0DD14D
:106740000B4B1B68002B03D09B68002B00D0984795
:10675000084B04211878084A05F072F870BDC0464D
:106760002843FF1F8464FF1F5E64FF1F8064FF1FB8
:10677000AC64FF1FB064FF1F60EA0000014B986823
:106780007047C0466464FF1F014BDB6818687047A0
:106790006464FF1F074B10B5DA6813680133136098
:1067A000054B1878FF2803D08021C90105F000FAB5
:1067B00010BDC0466464FF1F2843FF1FF7B50E00DD
:1067C00002F0C8F8051E1CD00E4B06621F78002F81
:1067D00000D10778AB791020019305F051F8041E21
:1067E0000FD0D0230380C73B8370019BE91DC3708A
:1067F0000622043005F0FCF821003800E66004F0C1
:10680000FFFEF7BD2643FF1F014B18787047C046B7
:106810008464FF1F054B002805D1054B1A78054BF2
:10682000002A00D1014B18007047C0467464FF1F56
:106830008464FF1F5E64FF1F014B58687047C046A9
:106840006464FF1F024B1868431E9841C0B2704732
:106850008864FF1F421E03000120152A03D9FF3B55
:106860005A425341D8B27047F0B51C0000230E00C5
:1068700085B0039002920B70029A934201D30020DC
:1068800019E0E55C5A1CD2B2002DF8D002985119DB
:106890008142F4DC0233DFB2A35C18000193FFF7FE
:1068A000D9FF002807D0013D019A0399EBB233705C
:1068B0008A4202D1E01905B0F0BDDB19DBB2DBE79B
:1068C00010B50C0002F09EF803001220002B03D03C
:1068D0002100588805F0BCF810BD000070B50E4DC1
:1068E00084006359002B15D0186A002801D004F0E9
:1068F000B7FE2B59586A002801D004F0B1FE2B597D
:10690000986A002801D004F0ABFE285904F0A8FED4
:1069100000232B5170BDC0469464FF1F1C4B70B503
:1069200004000E00150099420AD11A4B1B68002B77
:1069300001D1122070BD1B68002BFAD09847F9E7EF
:10694000154B994215D1134B1B68002B0AD01B68BD
:10695000002B07D09847002804D1104B1C70104B17
:106960001D70E7E729002000FFF7AAFF0028E1D10A
:10697000F3E7080001F0EEFF0028DAD003780320E7
:10698000A342D7D12900300005F062F8D2E7C04613
:10699000FEFF00009064FF1FFFFF00008D64FF1FDB
:1069A0008C64FF1FF7B50400808801F0D3FF002539
:1069B000A84203D00578A08802F008F81C4E33786E
:1069C000002B1FD0AB421DD11A4B28001978FFF7BE
:1069D00077FF002818D000233370A3790820A77808
:1069E000A688019304F04CFF011E0DD0D023037044
:1069F000CA3B8370019B477086808371280004F036
:106A0000FFFD01E0002DE8D1A0880B4B8200D35898
:106A1000002B01D0FFF762FF1721A088FFF768FD68
:106A2000A08801F027FDA08801F0FEFDF7BDC0465B
:106A30008D64FF1F8C64FF1F9464FF1FF0B587B047
:106A40001D000CAB1B88070001930DAB1B881420A5
:106A500002930EAB1B88160003930FAB1B880091AB
:106A6000049310AB1B88059304F00AFF041E1AD090
:106A7000D0230370CB3B47708370C6700622290079
:106A80000430002D11D004F0B3FF019B210063817D
:106A9000029B0098A381039BE381049B2382059BB7
:106AA000A37404F0ADFD07B0F0BD05F041F8ECE7CC
:106AB000F7B5009308AB1B8807000C200D001600EB
:106AC000019304F0DDFE041E13D0280001F042FF04
:106AD00000280FD00078D0232370C93BA370009BFF
:106AE00021002381019B6770A580E680638104F00B
:106AF00087FDF7BD014B1878EDE7C0462843FF1F1F
:106B000013B5040064890389C2888188C078009421
:106B1000FFF7CEFF13BD000010B5044C206800281D
:106B200003D004F09DFD0023236010BD9864FF1F77
:106B3000A122F0B5818892004A43384B384F1B6838
:106B400004009B189D2292009B18827989B01A60DC
:106B50003B68002B5FD01D78324B1B68002B04D0A4
:106B60005B68002B01D000209847260008363100D2
:106B7000E079FFF7B7FD237DE0710200E078049330
:106B8000638A29000393238A0293E3890193A388EC
:106B900000933300FFF752FFE378002B0BD1E2891B
:106BA000A379A18802920196E2792800009201223D
:106BB00001F0DAFEE0703B68002B20D0FFF7ACFF5D
:106BC000194D287800281AD0184B1978FFF778FE4D
:106BD000002814D02B78E67808200793A78804F0C3
:106BE0004FFE011E09D0D0230370CA3B467083704C
:106BF00087808671079804F003FD00232B7017210E
:106C0000A088FFF775FCA08801F034FCA08801F093
:106C10000BFD09B0F0BD064B9DE7C0463409FF1FD0
:106C20009864FF1FAC64FF1F8D64FF1F8C64FF1FFF
:106C30002843FF1FF8B5070008000E0001F08AFE88
:106C4000041E18D02620FFF78DFC051E00D12578E4
:106C5000062004F015FE041E0DD00021062204F0CB
:106C600067FFD0232370C23B21006770A370A6800A
:106C7000E8B204F0C5FCF8BDF0B585B001930AABED
:106C80001B78070002930BAB1B7808000D000092E5
:106C9000039301F05FFE061E22D0102004F0F0FDE9
:106CA000041E1DD01022002104F042FF2620FFF711
:106CB00059FC002800D13078D0232370C13BA37049
:106CC000009B21002372019B67706372029BA58069
:106CD000A372039BC0B2E3720C9BE36004F090FCD0
:106CE00005B0F0BDF7B50D00019001F033FE071EB1
:106CF00020D00E2004F0C4FD041E1BD02620FFF778
:106D000031FC061E00D13E78D0232380C53B0622ED
:106D1000A370F91DE01C04F06BFE019B2A00638147
:106D20000123DD401A401D40210022736573F0B23B
:106D300004F066FCF7BD0000F0B585B002901000CD
:106D40000D0017000A9E039301F004FE041E31D0CB
:106D5000029B002B2ED1039B02795B0724D51223C3
:106D600013430422002E08D10B99002905D10C9958
:106D7000002902D10D9900291AD01A430D9B2271C6
:106D8000002B00D0C9E0002E00D1CFE0002D00D0B4
:106D9000CCE0606A002801D004F062FC1C213000C5
:106DA00004F046FD606205E002239A430E33D7E704
:106DB00093432371654BBA00D458002C00D1AAE04C
:106DC000002E10D0236A002B03D11C2004F080FD7C
:106DD00020625E4BBA00D358186A002803D01C22E8
:106DE000310004F005FE0C9B002B12D0574CBB0069
:106DF0001D596B6A002B03D1162004F069FD6862EF
:106E0000BB00E358586A002803D016220C9904F0FE
:106E1000EFFD0D9B002B11D04C4DBC006659B36AA1
:106E2000002B03D1142004F053FDB0622B59986A53
:106E3000002803D014220D9904F0DAFD380001F087
:106E400089FD051E67D0414BBA00D358002B62D094
:106E50001A6A3420002A00D11C389A6A002A01D00C
:106E6000143080B20B9A002A01D01C3080B25B6AC9
:106E7000002B01D0163080B204F002FD041E4AD06F
:106E80001822002104F054FE2620FFF76BFB01902E
:106E9000002801D12B780193D0232370029B20007E
:106EA00063700A23294EA370039BBD00A371AB59E5
:106EB000A780196A1830002905D01C22A06004F0B0
:106EC00097FD200034307359996A002907D00300D8
:106ED00014221433E060029304F08AFD02980B9BA5
:106EE000002B08D003001C221C330B992061029355
:106EF00004F07EFD02987359596A002903D01622C6
:106F0000606104F075FD6B462100187904F078FB90
:106F10003800FFF7E3FC05B0F0BD10220D9B0D9982
:106F20001B69A018236204F063FD2CE70B9B002B68
:106F300000D13FE7012D00D03CE7606A002801D076
:106F400004F08EFB1C210B982AE7C0469464FF1FB7
:106F500010B5044C2068002803D004F081FB002306
:106F6000236010BD8864FF1F0B4B07B51A68002A09
:106F700001D100200EBD6946531C01201278073153
:106F8000FFF772FC0028F4D00278012310001840AB
:106F90001A42EED0EEE7C046A464FF1FF0B51F4FC3
:106FA00001203B6887B0002B25D09B78059300F02B
:106FB000B3FB002821D00A20FFF7D4FA04000B20ED
:106FC000FFF7D0FA164B05001E78731E9E413B68F2
:106FD000F6B2191DD878FFF757FB3B682900DA7A1B
:106FE000043303929A7901930292009033002000B7
:106FF000059A04F075FC07B0F0BDFFF7B5FF002857
:1070000005D00620FFF7AEFA04000720D8E70820D5
:10701000FFF7A8FA04000920D2E7C0468864FF1FE2
:107020008464FF1F70B50A4E040033780D00FF2BF7
:107030000DD0042004F024FC011E08D0D0230370DE
:10704000CE3B45708370C470307804F0D9FA70BDBF
:107050003843FF1F70B5040006200D0004F010FC3B
:10706000011E0AD0D0230370CD3B8370054B4470C2
:107070001B688580187804F0C3FA002C01D0FFF754
:1070800067FF70BD8864FF1FF8B5264F06003B6898
:107090000D001124002B05D10522234B1B78134230
:1070A00002D112242000F8BD204A10241268002AC0
:1070B000F8D01278002AF5D0DB0719D52B789A1E64
:1070C000012A1AD80C2004F003FC1324386000288D
:1070D000E8D000230A22437029000670023004F031
:1070E00087FCFFF75BFF041E0AD0FFF731FFD9E7EB
:1070F00000F012FB0028E1D1E4E7002BE2D0D0E75A
:107100000B4B1B78032BCDD11D20FFF72BFA094B1E
:1071100018800028C6D0084B04211878074A04F0CC
:107120008FFBBFE78864FF1F8564FF1FA464FF1FF8
:107130008464FF1F8264FF1FB064FF1F60EA0000C9
:10714000F7B50193194B14001A78052306000F00B8
:1071500012201A4221D0012920D1154B1D68002D83
:107160001BD002201F2C18D8002C02D0019B002B12
:1071700013D0104B1F221E706E1C0021300004F033
:10718000D7FC01992200300004F032FC31002000CD
:107190002C70002F06D004F0D3FAFEBD064B12204F
:1071A0001D68DCE704F09CFAF7E7C0468564FF1F22
:1071B000A464FF1F3843FF1FA064FF1FF8B50F4EE4
:1071C00012243368002B17D01B780F3C834213D155
:1071D00000250B4F0221387804F022FB094B0421D3
:1071E00038781D8004F01CFB074B28001D80336895
:1071F0005C7004F085FB04002000F8BD8864FF1F6C
:10720000B064FF1F9C64FF1F8264FF1F70B50128DC
:1072100023D11B4C2388002B03D01A4A1578002D4C
:1072200007D0194B1B68002B02D01878FFF7C6FF58
:1072300070BD3B2B02D93C3B2380F9E7134E022162
:10724000307804F0EDFAFA222388920002215A43A2
:10725000307804F065FA2580EAE70B4B1B68002BB9
:10726000E6D00B4B1B785B07E2D5084B0221187860
:1072700004F0D6FA0022024B1A80FFF769FED7E726
:107280009C64FF1F8064FF1F8864FF1FB064FF1FA2
:107290008564FF1FF8B51E4D2868002803D004F050
:1072A000DFF900232B601B4E3068002803D004F068
:1072B000D7F900233360184F05243B78180020408D
:1072C000234221D0154800F02BFA3B78234213D0FB
:1072D000202004F0FDFA2860002813D0202200218D
:1072E00004F026FC202004F0F3FA041E306005D0E0
:1072F0002022002104F01CFC002004E0286804F097
:10730000AFF92C601320F8BD00F00AFAF4E7C0468C
:10731000A464FF1FA064FF1F8564FF1F2C43FF1F91
:1073200010B50A4C23681A1E0ED0002808D101306F
:10733000587004F0E5FA002805D02368002B02D02D
:107340000021FFF787FE0122100010BD8864FF1F97
:10735000F7B5274E050033680191181E21D05C78DF
:10736000244F012C30D1FFF7FFFD002825D020004D
:10737000FFF7F8F80400412814D91F4B02211878B0
:107380001E4A04F05DFA1E4B3C3C1C80022233680E
:107390005A703B78002B14D128000199FFF75AFE50
:1073A0000120FEBDFA2292004243002AEED0124B89
:1073B0000221187804F0B4F9E8E7FFF7D3F80200E7
:1073C000F3E700233B70EBE73B78002BE8D1032089
:1073D00004F056FA011E08D0D0230370CC3B457050
:1073E00083703368187804F00BF9FFF7B1FDD7E725
:1073F0008864FF1F8064FF1FB064FF1F60EA000005
:107400009C64FF1F10B51749838802008B4220D06F
:1074100011D815498B4217D0144900205B1899B236
:10742000012907D8926811785A425341D8B2FFF720
:10743000F9FD012010BD0E4A00209B1807229BB2C7
:107440009A424041C0B2F5E783681878FFF768FFB9
:10745000F0E7836899785A78090218781143FFF7A2
:1074600077FFE7E70A20000006200000F8DFFFFFB3
:10747000AFDFFFFF014B18707047C0463943FF1F55
:1074800010B5064C207001F041FA207804F008F99C
:107490000521207800F062FD10BDC046B064FF1FDA
:1074A0000BB273B50D00002B00DBC4E0884B1878DD
:1074B00004F026F9041E0ED00378912B0FD0A22BD6
:1074C00000D1A1E0834B1878FF2852D0210004F0AE
:1074D00097F800284DD180200002684076BD43789F
:1074E0000F2B76D013D8052B70D00E2BEAD18088C5
:1074F000794B98422BD8794B98421BD8784B9842BD
:10750000E0D1A3681878591CFFF774F838E03E2BD7
:10751000D8D18378032B74D06CD8012B6ED0022B7A
:10752000D0D1704B1B68002B23D05B68002B20D080
:1075300098471EE06C4BC0180C28C3D804F048FBD9
:107540001DC2C2150BC20B0B0B3223C23C00674B92
:10755000C0180728B6D8664B1B68002B09D01B68DB
:10756000002B06D0200098470AE0A3681878FFF7A0
:10757000C7F8200004F004FBADE7A068FFF762F84D
:1075800000289FD0F5E7A3681B78002BF1D0554B5E
:107590001B68002BEDD01B68002BEAD0210055485A
:1075A0009847EDE74F4B1B68002BE2D01B68002B80
:1075B000DFD021005048F3E7504B1B68002BD8D098
:1075C0005B68002BD5D021004348E9E7FFF7EAF9D3
:1075D000CFE780884A4B984203D04A4B984200D06C
:1075E00070E7464B1B68002BC3D05B68002BC0D0F4
:1075F0002100D5E7153B012BBBD963E7FFF798FACC
:10760000B7E7FFF77DFAB4E73F4B1B78042B07D1B0
:1076100000236A4613800179408800F0C5FCA8E782
:10762000364B1B68002BA4D05B68002BA1D0010057
:10763000364898479DE7012421420AD0294B1B6810
:10764000002B04D05B68002B01D00020984701205C
:1076500043E78B070AD5264B1B68002B04D05B68D9
:10766000002B01D020009847022036E70421280093
:1076700008400D4200D131E7254E3388002B21D040
:10768000013B9BB23380002B1AD1FFF7DBF80028B7
:107690000AD0204B1C70164B1B68002B04D05B6873
:1076A000002B01D020009847FFF7C6F8694601F08B
:1076B00001FD6846FEF7FEFF1D20FEF753FF3080F8
:1076C00004200AE7024B187804F0AAF8F8E7C0464D
:1076D000B064FF1F3943FF1F0E200000012000008F
:1076E00009100000A864FF1FFEDFFFFFAFDFFFFFF0
:1076F000AC64FF1F0C2000000B2000009064FF1FF3
:107700000D200000132000008564FF1FFFFF000014
:107710008264FF1F8064FF1F10B501F09BF910BD4C
:10772000014B18607047C046AC64FF1F0B880020F7
:10773000162B01D817230420014A13807047C04636
:107740005A64FF1F00207047074A030011888142D6
:1077500007D091880020994202D101308000101892
:1077600070470020FAE7C046B864FF1FF0B58F7875
:1077700006000D00C5B01E2F15D1FFF7E5FF051E51
:1077800003D10024200045B0F0BD00223B003100B1
:10779000C078009200F0B2FB0400A81C00F0D2FBFD
:1077A000FF23EB70EEE7264B062403931B78FF2B99
:1077B000E8D0182FE6D87B08224A013BDB00029272
:1077C0009A589446002ADDD0029AD3185B68002BA1
:1077D000D8D00878002802D14B78012B02D106249A
:1077E000122FCFD107AFAB88697800976446AA689B
:1077F000A047041EC6D1AB78029A5B08013BDB00B0
:10780000D318390030005B689847041E0BD1AB7861
:10781000042BB6D0039A310010782200009700F0B4
:107820006DFB0400AEE76A78002AABD1AA7805A9FF
:107830003B88087130000A704B80FEF747FBA0E7D9
:107840003C43FF1FE8BD00111D4B37B505009842B2
:107850000BD000290AD1FFF777FF002805D119487E
:10786000FFF772FF002800D0058037BD01291AD12B
:10787000FFF76AFF041EF8D001235B420380A37860
:10788000FF2BF2D0FE2B07D00023E07814220093C8
:1078900029001E3300F032FBA01C00F053FB012333
:1078A0005B426380E1E70229DFD1013901F0BEF8D4
:1078B0000028DAD12800FFF747FF041EDFD1D4E704
:1078C000FEFF0000FFFF0000022210B5074B5242EE
:1078D0001A80074801325A809A80DA8000F07EFAD6
:1078E000044801F025F8002010BDC046B864FF1F11
:1078F0006D770011497800110388F7B50400002B5B
:1079000002D102252800FEBD4268022113782548D5
:107910005268FEF7A5FD00282ED0234F01253A8896
:10792000002AEFD0802321885B0201259B1A99420F
:10793000E8DC0C2003F0CCFF061E31D03B88228807
:107940009C4600231800019561469DB2491989B2F1
:10795000AA421BD8002801D062443A80002330009C
:10796000082208C0210004F043F8104A1368002BD5
:1079700013D100251660C5E76268022113780C4810
:107980005268FEF76DFD0028C7D1BAE760681D0197
:107990004019418101330198D6E71A001B68E6E7D8
:1079A0001325AFE756BE00113A43FF1FB464FF1F13
:1079B00054BE0011014B18707047C0463C43FF1F76
:1079C00014230A0010B51A40194204D001221021D4
:1079D00001F048F810BD4B06F9D40120884340005F
:1079E000F8E710B514008B0604D50122102101F030
:1079F00039F810BD08230A001A40194202D14BB2CF
:107A0000002B0FDA102101F02DF8002808D02300F8
:107A1000F2331B78002BECD0F1342378012BE8D122
:107A20000020E6E703208907FAD4E2E7F0B51F005B
:107A3000184B85B01C68019002910392002C27D14D
:107A4000200005B0F0BDA5683301ED186B89019ADF
:107A5000934211D3029A93420ED8002F04D10A9B6D
:107A6000002B10D12C00EBE73B002978039A6868C3
:107A7000FEF7F6FC0028F2D10136B6B2A388B34275
:107A8000E1D82468DAE7A3680A9A5B891380E9E7FA
:107A90000026F3E7B464FF1F37B50C000A88498855
:107AA0000123914217D3002A15D0651D23792A009E
:107AB00002210A48FEF7D4FC102300280BD02379BA
:107AC0006188208800242A000094FFF7AFFF0A2372
:107AD000A04200D0230018003EBDC04656BE001193
:107AE00013B50A0008884988012388420BD800286A
:107AF00009D00024137905320094FFF797FF0A2379
:107B0000A04200D02300180016BD13B50A00088853
:107B10004988012388420BD8002809D00024137912
:107B200005320094FFF782FF0A23A04200D0230011
:107B3000180016BDF0B58BB003904A8808880E0077
:107B40000123824255D3002853D00023012704ACDF
:107B500023700022718813000092FFF767FF051E53
:107B60003ED02078002835D12B78022B18D16770B1
:107B70006A8983000130E31880005A806968022214
:107B8000201803F035FF23780133DBB22370042B78
:107B900019D93B006889013080B2002BD9D01FE091
:107BA00002236370122358436A89231804305A80D1
:107BB00069681022201803F01BFF23780133DBB221
:107BC0002370002BE5D10C4A6B899B185A42534114
:107BD000DBB2DFE76378012BE4D12B78022BC7D02F
:107BE00022780A23002A04D021000398FEF798F98E
:107BF000002318000BB0F0BD0100FFFF0F4BF0B5E4
:107C000004001868002816D083685D89A54207D84B
:107C10008288AE18B44203DA12019A18934201D155
:107C20000068EFE71E005F891036A74204D10029E3
:107C300000D00D801800F0BD3300EFE7B464FF1FE3
:107C400070B505000C0008880021FFF7D7FF03007E
:107C50000120002B04D022002800197AFFF7C1FE72
:107C600070BDF7B50C00002501902300EE331B78A2
:107C7000AB4201D800200AE06B00E65A0021300038
:107C8000E718FFF7BBFF002802D126800130FEBDB8
:107C9000017A0198FFF794FE002802D03B882380E8
:107CA000F5E70135EDB2E0E710B5040008880021E2
:107CB000FFF7A4FF03000120002B03D02000197A56
:107CC000FFF77EFE10BD0000054B1B68002B01D1A5
:107CD000180004E09A6852898242F6D19888704769
:107CE000B464FF1FF0B50E27002687B0039302ABE4
:107CF000FF183E8005001F4B40891400984207D0B2
:107D00002B78013000976A6880B2FFF78FFE06007B
:107D100002212B7818486A68FEF7A2FB00280FD0D2
:107D20006C892000FFF7D0FF002802D0013C041925
:107D3000A4B2039B002B00D01C80300007B0F0BD24
:107D400002212B780D486A68FEF78AFB0028E7D1EC
:107D500002212B780A486A68FEF782FB002807D0C8
:107D6000002EDED03B88A342DBD17489013CDFE7E3
:107D70006C89DEE7FFFF000056BE001154BE001103
:107D800052BE001110B50C00FFF7DEFC030002200C
:107D9000002B0AD0002C00D023609B781720FE2BEC
:107DA00003D00138FF2B00D1002010BD73B50D00AA
:107DB00001A904001600FFF7E5FF172805D0002EE3
:107DC00004D129002000FEF727F976BD01221021F9
:107DD000200000F047FE0028F3D0F6E7014B1860C2
:107DE0007047C046C464FF1F37B56B469D1D010038
:107DF00004000222280003F053FD2B88B02B0ED183
:107E00002379122B09D12300FA331B78012B06D1D9
:107E10000121608800F0E0F801E01B2BF8D037BDAD
:107E200010B5054B0421187000F098F8FFF74CFDD1
:107E3000FEF770FB10BDC046C864FF1F0020F0B500
:107E40000BB20F0087B0834234DA274B187803F067
:107E500057FC051E2BD00378A02B25D103AE310093
:107E6000FEF7E4F8041E0BD1B378DB0724D51F4BD3
:107E700006341B68002B03D0310068889847040043
:107E8000A868002801D003F0F3FC002C08D1184AA0
:107E9000039B1340174A934206D0B3781B2B03D0A1
:107EA0000121688800F098F8280003F069FE80201E
:107EB0000002784007B0F0BD0F4B1B68002B10D0BC
:107EC000310068889847041EDAD07378002BD7D128
:107ED000B27801A90A704B800C716888FDF7F6FF33
:107EE000CEE70624F1E7C046C864FF1FC064FF1F49
:107EF00000FFFF0000011200C464FF1FF7B50190EE
:107F0000FC200D0017001E0003F0BAFC0400132033
:107F1000002C12D0B02320002370089BF42267703D
:107F2000658026710830002B08D0190003F060FD31
:107F30002100019803F064FB0020FEBD089903F0C6
:107F4000F7FDF5E710B5041E06D00078FD2803D82C
:107F500003F02EFCFF23237010BD00000A1F93B214
:107F600010B504000220032B05D882400020024BEC
:107F7000D1529B189C7010BDE864FF1F0B8870B530
:107F8000043B04000D000220032B0BD8012120002C
:107F900000F04CFD03001420002B03D0290020002A
:107FA00000F0DEFB70BD000007B51300034A00922D
:107FB0000A00012100F02CFC0EBDC046E581001135
:107FC00007B5019203220092024B0A00122100F031
:107FD00049FC0EBD6382001107B56B4601AA1180F2
:107FE0000449D88008780633012802D1190003F02B
:107FF000AFFB07BDC964FF1F0C4B10B51870002301
:10800000FF210B4A1380138193819380094A538087
:108010001370517293819372D174D3821375517717
:1080200003F026FB00F0FCF910BDC046F864FF1F0A
:10803000E864FF1FCA64FF1FF0B58DB06B460020D7
:1080400003910C229B5E834200DBB0E05D4B18780D
:1080500003F056FB051E00D1A4E00378902B00D05E
:108060009DE006AF01004688380000F013FA7968F9
:108070000400002900D19CE03B88052B6ED13B8990
:10808000032B1CD905AC200000F0A2F86288172A47
:1080900061D83989131D994231D179682378043127
:1080A0000291D90738D5607800F08EF9071E06D006
:1080B000002303712378012B08D0132B23D0A86849
:1080C000002800D178E003F0D3FB75E062880299C4
:1080D00009A800F0A6F80290380000F08BF909AA70
:1080E0002378387A0192002231000092029A00F03F
:1080F00012F9380000F064F9029B002BDFD0300049
:1081000000F080F9DBE70378032BD8D1628802996D
:1081100009A800F0D6F8DEE7122B13D1029909A8BE
:1081200000F0B5F8021EEAD127498B88002BC6D093
:10813000887909A92378019161780091310000F0D4
:10814000EAF8BCE7002302AA93833000617809AA09
:10815000FFF72AFFB3E71D4B0993F6E7042B02D084
:108160009A1F012AABD8184A043B9B00995A002950
:10817000A5D0D218907831003A0000F0AEF800286F
:108180009DD13B88042B03D001213000FFF724FF51
:10819000012C04D1A868002801D003F069FB280055
:1081A00003F0EEFC8020039B0002434018000DB05A
:1081B000F0BD012800D182E701213000FFF70CFF5C
:1081C000EDE7C046F864FF1FE864FF1F01001700D9
:1081D0000B7803704B784370CB788A781B0213437B
:1081E000438070470A88030002700A88120A4270AE
:1081F0000A88012A06D14A8882704A88120AC27007
:108200000420704702208242FBD14A8804309A70D1
:108210004A88120ADA708A881A718A88120A5A7190
:10822000EFE710B50400012082420CD94B780A78A0
:108230001B0213432380834206D1CB788A781B022A
:1082400013436380002010BD022BFBD1CB788A78CA
:108250001B02134363804B790A791B021343A380EB
:10826000F0E70B8803700B881B0A43704B88837000
:108270004B881B0AC3708B8803718B881B0A437160
:10828000CB888371CB881B0AC37108207047030019
:108290000120082A14D14A780878120202431A8071
:1082A000CA788878120202435A804A790879120201
:1082B00002439A80CA798879120202430020DA8048
:1082C000704710B504000120022A05D100204B7828
:1082D0000A781B021343238010BDF8B50600102056
:1082E0000F00150003F0CCFA04000120002C0ED082
:1082F000A0230C22290023806780201D002D07D099
:1083000003F076FB2100300003F07AF90020F8BD7D
:1083100003F00EFCF6E7F7B51E00009008AB142042
:1083200017001D78019103F0ABFA041E12D0A223AE
:108330000370019B47704380099B057146710C22B5
:108340000830002B07D0190003F052FB21000098E1
:1083500003F056F9F7BD099903F0EAFBF6E737B5E4
:10836000041E0FD04388002B0CD00025C188132396
:10837000007A172201950095FFF7CDFFFF23658056
:108380006372257037BD000010B50C4904004A889F
:10839000002A09D08B89002B05D00020CB8A02222D
:1083A000834201D010BD012213000A204343002064
:1083B0004032C854C81842800472F3E7CA64FF1FF1
:1083C0000023438003707047094B00211A0010B549
:1083D0005C88002C06D01C79844203D10A234B43CD
:1083E000D01810BD01310A330329F1D10020F8E77C
:1083F000CA64FF1F10B50400407A03F0D9F9FF23C7
:10840000637210BD7047043010B580B203F028FBD2
:10841000002803D00421494203F002FC10BD0000F3
:1084200070B50025104CA0682580A581A580A842C4
:1084300002D003F01DFAA56000250C4C0C4B606DBA
:108440001D80230058331D70A84202D003F010FA9B
:10845000656500256068002801D003F009FA013540
:1084600008340A2DF6D170BD9065FF1F3465FF1FDB
:108470008465FF1F70B5041E09D1054D2880A881B1
:10848000A880A868002802D003F0F2F9AC6070BDA3
:108490009065FF1FF0B54B8885B0019300234360C2
:1084A0000A7905000F00022A00D07BE0CA88032A5F
:1084B00017D98B685E7819783602DC78D8790E4344
:1084C00099781B7A24021B020C43034353495BBA7D
:1084D0000B80331D93421ED1042C04D0631F022B4A
:1084E0000ED9012015E0019A4D4B1201D35A002BF1
:1084F00006D00198FFF7BEFF4A4A136901331361A2
:108500000421B8682E812C80494203F089FB686001
:10851000002005B0F0BD434D042C06D0631F022B94
:108520000FD9EB680133EB60DBE7019A3C4B12019A
:10853000D35A002B05D00198FFF79CFF2B6901331C
:108540002B61374B30000293019B029A1B01019370
:10855000002301998C468B52130063449C80039343
:108560009E81FFF750FF039B041E986016D00421E4
:10857000B868494203F054FBFA880100043A20002D
:1085800003F036FA0199029AFB888A5A043B9B1839
:10859000029A8B522B6801332B60A2E7AB6901333F
:1085A000AB619EE71E4B0293019B1E01029BF35A97
:1085B000002B2DD002998C19A068002828D0012A00
:1085C00026D1FA889B189BB27352A189994217D37E
:1085D0009B1AC018B96803F00BFA029BA289F35AE0
:1085E000934200D07DE700222B81A3882B80A368D3
:1085F0006B60029BF2520B4A53680133536070E781
:10860000084A9368013393600198FFF733FF68E7E6
:10861000044A536901335361F6E7C046FA64FF1F09
:108620009065FF1F0065FF1F70B5051E15D10B4C2F
:108630000B4B1880230058331870606D002802D04F
:1086400003F016F96565250050356068002801D0F3
:1086500003F00EF90834AC42F7D170BD3465FF1F4A
:108660008465FF1FF0B51700A12285B09200019329
:108670004243394B06001B680C009B18D933FF336B
:108680001D78FDF741FF0430854204DD3000FDF721
:108690003BFF0430C5B2BD4207D33A000021300091
:1086A000019B03F04DFA05B0F0BD2900380002F03F
:1086B000BFFF2300C6B250331E700393019B2900F5
:1086C0006365380003F054FACBB20293002B02D05A
:1086D000039B01361E7000262300503303931B7842
:1086E000B34204D8606D002831D10020DBE7029A44
:1086F0002800002A04D0013B1000B34200D028001B
:10870000F700E719387003F023FA786000280ED0DC
:108710003A78019903F06CF9019A3B780136D31845
:108720000E4A0193D369F6B20133D361D4E7039BB8
:1087300018706065A74205D1084A1320D36A013337
:10874000D362B0E7606803F093F80834F2E703F00F
:108750008FF800236365C8E73409FF1F0065FF1F1A
:10876000F7B50D0007000421686803F059FA2B895A
:10877000040003702B891B0A43702B8883702B889D
:108780001B0AC3702E8902250436F6B2F42E15D8C2
:108790001B4B9F4214D10C2003F072F81135011EBF
:1087A0000CD0902303708E3B0371043B4380154B28
:1087B0008460C680187802F023FF00252800FEBDE3
:1087C0005C237B43104AD3180093583301931B78E2
:1087D000002B0FD10300320038000099FFF742FF51
:1087E000019B05001B78002BE8D13800009902F0AE
:1087F0004FFFE3E7054A0725536A01335362DDE77C
:10880000FEFF0000F864FF1F3465FF1F0065FF1FB7
:10881000F0B587B0009017200F0016000193FFF706
:10882000F2FD1325041E19D00C98031E02D00199E5
:10883000201D9847030AE370052302AAA0700430A4
:10884000908127700098667003A993800494FFF7C5
:1088500087FF051E02D0200003F00AF8280007B0A9
:10886000F0BD0000F0B587B01F000CAB1B78039182
:10887000059301210DAB06001C78049200F0D6F898
:108880001425002821D02000FFF77EFD0135041EAD
:108890001BD01149059B0A7803700132D2B2131E16
:1088A000C68001D101231A000B7022713000049B95
:1088B00003990097FFF7ACFF051E09D123002100A3
:1088C0000648074A093302F06BFF280007B0F0BDE5
:1088D000002363802370F8E7FC64FF1F5F830011AF
:1088E00030750000F8B505000E00064C064F2368F1
:1088F000002B02D03100280098470434BC42F6D146
:10890000F8BDC046A065FF1FB465FF1F0123064ADE
:108910005B425380002313715362044A1360536017
:108920009360D36013617047B465FF1FA065FF1F9C
:108930000200002310B506499C000859002801D107
:10894000625010BD0133052BF6D11320F9E7C04664
:10895000A065FF1F034A5388181A434258414042FA
:1089600010407047B465FF1FF0B585B002930AABA5
:108970001F780CAB1B88009008000E000192039337
:10898000FFF7E8FF05001120002D1BD10E48FFF76F
:10899000E1FF04001520002C14D006220B99A771CA
:1089A000E01D03F025F8019B30002371029B290094
:1089B0006371009B66802370039B6562E381FFF710
:1089C00091FF280005B0F0BDFFFF000010B5FFF7D4
:1089D000C1FF04000220002C12D060880121FFF7A3
:1089E00081FF606A002801D002F03AFE28220021AF
:1089F000200003F09DF8012300205B42638020717A
:108A000010BD000030B5074A074C558801001378A7
:108A10000020A54204D05B1A59424B4158421040F5
:108A200030BDC046B465FF1FFFFF0000084A10B507
:108A300001230C00904208D0FFF78CFF031E04D0E6
:108A4000037923405A1E9341DBB2180010BDC04683
:108A5000FEFF0000024B1879431E9841C0B27047D8
:108A6000B465FF1F70B504000D001600FFF772FF1C
:108A7000002804D10D4B9C4200D0143070BD416AD7
:108A800003790520002907D012221A40102A02D1AA
:108A90000520002EF2D10F20DB06EFD5897E0C20B9
:108AA000A9428941494249420840E7E7FEFF0000E8
:108AB000030010B5002800D110BD0348034A4188C7
:108AC0009142F9D09847F7E7B465FF1FFFFF000018
:108AD000002330B5C45CCD5C6C40D4540133102B02
:108AE000F8D130BD0F23002210B5C45C64002243CE
:108AF000CA54C25CD209013BF7D210BD020001008A
:108B000010B52032103103F073F810BDF0B58BB002
:108B10000390102005931700049102F0D9FE0090F5
:108B2000102002F0D5FE009B13240190002B05D0ED
:108B300000280CD11324009802F092FD019B002B19
:108B400002D0180002F08CFD20000BB0F0BD102008
:108B500002F0BEFE0600102002F0BAFE132405004B
:108B6000002E00D1AEE0002819D01022002102F022
:108B7000DFFF32002900039803F03AF8041E0ED1FB
:108B800033787F2B51D830000099FFF7ABFF009B63
:108B90001B787F2B53D801990098FFF7A3FF300073
:108BA00002F05EFD002D02D0280002F059FD002CDD
:108BB000C1D1102002F08CFE0600102002F088FEC9
:108BC0000290002E7CD0002878D03A000F3223008B
:108BD0000125121105D00F333B4015B25A425341C3
:108BE0001BB26A1E1201002B33D0049BD2B298181C
:108BF0000099029AFFF76CFF013D1022002130001E
:108C000002F096FFADB2049F2D017D19AF4242D014
:108C1000002C33D0300002F023FD029B002B00D14A
:108C200089E7180002F01CFD85E729003000FFF7F6
:108C300059FF28002549009AFFF74AFFA7E72900B6
:108C40000098FFF74FFF28002049019AFFF740FFE7
:108C5000A5E70F210F4004998A18D9B28F4208D98D
:108C6000D15C06A819540133102BF6D1029A019950
:108C7000C0E7791A48424141C901F2E739003000A2
:108C800006AAFFF725FF3200039806A902F0B0FFFD
:108C900010370400BAE7002CBCD13000029906AAB4
:108CA000FFF716FF320006A9039802F0A1FF082281
:108CB00004003100059802F09BFEABE71324A9E7FE
:108CC0001324AAE7002800D06EE733E75CBE00114A
:108CD000F0B58BB00F0016000225009000283FD0A1
:108CE000002A3DD00B1DDBB21800029302F0F0FD0C
:108CF0001135041E34D0FDF747FD05003A000099F8
:108D0000201D02F075FCEBB20393E3702B0CDBB279
:108D10002F0A00936370FFB22B0E2370A77001938C
:108D2000FDF72CFD1022010006A802F061FC2100D5
:108D3000029A04AB06A8FFF7E9FE051E0DD1039BBE
:108D400008223370009B04A9B370019B7770F37005
:108D5000301D02F04DFCFDF71DFD200002F080FCEF
:108D600028000BB0F0BDF0B58FB00D00149E03903D
:108D700004920593002A03D1022420000FB0F0BD15
:108D8000002EF9D00398FFF7E5FD1424071EF4D058
:108D90007278337812021A43B3781B041343F278C3
:108DA00012061A43036A0192934201D30133E3D1BD
:108DB000002D03D03B7901249B07DED5082200213A
:108DC00006A802F0B5FE059B13240433DBB218009D
:108DD000029302F07DFD051ECFD0059A0499043060
:108DE00002F006FC04223100280002F001FC3900E8
:108DF000102210310AA802F0FBFB2900029A06ABF0
:108E00000AA8FFF783FE041E0FD1082206A908A8AE
:108E100002F0EEFB0822311D08A802F0A9FD01288E
:108E200007D101990398FDF7C9FC280002F018FC4E
:108E3000A3E70124F9E7000070B51C4C0500236886
:108E4000181E10D0002D14D11A78002A0CD1981CAD
:108E5000083202F0CDFD02F0B3FC0135002808D144
:108E600023681D70012070BD0A331800082202F02B
:108E7000BFFD2368002BF5D0122002F001FD061E75
:108E80000DD0C123216803704570023110220230D9
:108E900002F0AEFD23683100587802F0B1FB206883
:108EA00002F0DEFB00232360DCE7C046DC65FF1F29
:108EB000F8B504002020FDF755FB0D4EA700BB5967
:108EC0000500002B0DD000280BD0D878FF2809D141
:108ED00008492A000C55F35907480333611802F07A
:108EE0005FFCF8BD290002F073FC0028F0D1F8E720
:108EF000F865FF1FE065FF1F09A1001170B5064D61
:108F000084006359002B05D0D87802F051FCFF2271
:108F10006359DA7070BDC046F865FF1F70B5060072
:108F20008CB00C00150000213022684602F000FED3
:108F300031001022684602F05BFB1D202100032255
:108F4000684402F055FB6846FFF7D8FD2D21040068
:108F500003222800694402F04BFB20000CB070BDD6
:108F6000F0B50700160097B001931CAB1D783022B6
:108F70001EAB00910AA800211C7802F0D9FD102236
:108F800039000AA802F034FB1022002102A802F0E6
:108F9000CFFD0722310002A802F02AFB072202AB14
:108FA0009818631E9C41019902F022FB02AB9C734E
:108FB0002B005A1E934102AAD3730021102206A847
:108FC00002F0B6FD06221D9907A802F011FB1A2037
:108FD00002ABC01806221F9902F00AFB102200996A
:108FE0000EA802F005FB102202AB0EA908781C782F
:108FF000013A6040D2B2087001330131002AF5D144
:109000000AA8FFF77BFD102212A904000EA802F0A7
:10901000EFFC102206AB0EA908781D78013A6840D3
:10902000D2B2087001330131002AF5D10AA8FFF746
:1090300065FD044310222098E4B212A902F0D8FA88
:10904000200017B0F0BD70B50E0014008CB0010008
:10905000102268461D0002F0CBFA3100082204A855
:1090600002F0C6FA2100082206A802F0C1FA6846FA
:10907000FFF744FD04001022280008A902F0B8FA06
:1090800020000CB070BDF8B506000D0000243719A3
:10909000AC4200D3F8BD02F0C3FA030A3B70631C74
:1090A000DBB201379D4203D90234F054E4B2EEE75B
:1090B0001C00EDE773B506000C000225002819D04E
:1090C000002917D0032101A8FFF7DDFF6B469A792D
:1090D0003F231A40013313436A463000937101A9BC
:1090E0002200FFF71BFF051E04D10322E01C01A98B
:1090F00002F07EFC280076BD03785807DA08C00F1E
:10910000D20080009B0710439B0F1843C0B27047EA
:1091100007230B40C908C9000B43037070470000C8
:1091200070B50400FFF7EAFE134DA4006359002B4D
:1091300021D0186A002801D002F092FA2B59986EBB
:10914000002801D002F08CFA2B59D86E002801D0EB
:1091500002F086FA2B59186F002801D002F080FA2D
:109160002B59586F002801D002F07AFA285902F0E2
:1091700077FA00232B5170BDF865FF1F0E4B80005E
:10918000C35870B50C00002B0FD09D68002D0CD07B
:109190002B78201D0B706B784B70A97CFFF7B8FF04
:1091A0002B7E23726B69E36070BD102200212000CA
:1091B00002F0BEFCF8E7C046F865FF1F014B1860DF
:1091C0007047C046F465FF1F074A030080008258BD
:1091D00010B5002A06D0D088984203D1012901D1C8
:1091E000FFF79EFF10BDC046F865FF1FF0B5264E85
:1091F00095B087000B93BB590500099112200A9284
:10920000002B31D0D888FFF7A5FB04001420002CD8
:109210002AD0280010A9FFF7B1FFBB591E781D6A9C
:10922000002E23D00895FDF7EFFA07000020FDF788
:10923000F1FA0790A379E61D069310AD0CA90898E2
:1092400000F0E2FA0EA9280000F0D7FA0B9B0A9969
:109250000493069B09980293079B0396019300973A
:109260000EAB0CAAFFF77CFE15B0F0BDFDF7CCFAF3
:1092700006903000FDF7CEFAE31DA779079310ABF7
:1092800006000893DAE7C046F865FF1F30B50C4CBE
:1092900085002A59030085B00120002A0ED018004D
:1092A0006946FFF76BFF2B591A78D888054B002ABF
:1092B00000D1054B6A46072100F0D9FB05B030BD4F
:1092C000F865FF1FFB9700110998001130B5094C94
:1092D0008500295985B010226846253102F088FBA7
:1092E0002A591121044BD0886A4600F0C0FB05B012
:1092F00030BDC046F865FF1FA598001130B5094C78
:109300008500295985B010226846353102F070FB7E
:109310002A591121044BD0886A4600F0A8FB05B0F9
:1093200030BDC046F865FF1FE3980011F7B54D4FFB
:1093300086001020F4590D0002F0CAFAF359206299
:10934000186A132200286CD0033A29009C6802F0A6
:109350004FFBF3591A780192002A58D11E6A227DD8
:10936000317B944651400122019F114201D1674651
:109370001740217D914339432175377B4F40BC46CF
:1093800060460027800701D44F08174001210220C2
:109390008F40227D82433A432275377B5740BC463B
:1093A00060460027400701D497080F400420227D23
:1093B000BF0082433A432275627D0027944660468F
:1093C000727B42400A4201D167460F400121627D13
:1093D0008A433A436275777B5740BC466046002714
:1093E000800701D457080F400220627D7F0082432E
:1093F00017436775767B00227E40760701D4BA0852
:109400000A400426617D9200B1430A4362756A787E
:10941000002A08D06278002A05D005220533DA77C1
:1094200000221000FEBD04222979114205D1A17C41
:10943000114202D10533033AF1E7019A21782C78E1
:10944000002A02D10A002100140018220429E8D8B9
:10945000042CE6D805206043034A05331218525CF9
:10946000DDE7C046F865FF1F6CBE001110B50A00AD
:109470001121024B00F0FBFA10BDC0463F990011CC
:109480000B0030B587B001AD2B806B460400110096
:10949000981D082202F0ACFA2A000B212000024B92
:1094A00000F0E5FA07B030BD6799001110B50A0069
:1094B0001121024B00F0DBFA10BDC046BB99001130
:1094C00013B50B0011006A4613706B4604000622A8
:1094D000581C02F08DFA6A4608212000014B00F06A
:1094E000C6FA13BDDB99001110B50A001121024B19
:1094F00000F0BDFA10BDC0462B9A00117FB50500E3
:109500000B4BAA00D4580800002C0FD0666F237FA5
:10951000E28821780396266F0296E66E0196A46E85
:109520000094FDF709FC2800FFF7FAFD7FBDC04657
:10953000F865FF1F10B51721FFF7E0FF10BD000011
:1095400070B50A000D00064B0221040000F08FFAEE
:10955000060029782000FFF7D1FF300070BDC0461B
:109560000B99001170B586B000236A4613708368AA
:1095700004001D78681E0A2859D801A902F0E8F9EC
:10958000060633373B3F43474B4F5300180000F06C
:1095900042F9062312284BD000281BD16088FFF720
:1095A000D9F90823002813D04279002A47D1264B45
:1095B0001A78072312070BD5244B1A680723002AB1
:1095C00006D01668002E03D0290001AAB047030078
:1095D0006A4613706B461B786088002B2AD1FFF710
:1095E00067FC06B070BD180000F06CF9D4E71800F5
:1095F00000F087F9D0E7180000F093F9CCE71800E5
:1096000000F0ADF9C8E7180000F0C3F9C4E718008E
:1096100000F0F6F9C0E7180000F0F6F9BCE7180012
:1096200000F013FAB8E7180000F013FAB4E70723C4
:109630006A46137069466088FFF782FFD1E7052309
:10964000012AC5D1024BB8E78564FF1FF065FF1FF3
:10965000F465FF1FF8B52C4F8600F35904000D0088
:10966000002B40D0DA8882423DD15A78062A33D185
:109670001A78002A2ED0012099681A6A097D0142C1
:1096800006D0157B054203D007225A700120F8BD91
:109690000220014204D0157B054201D00922F4E7E3
:1096A0000420014204D0127B024201D00B22ECE7DD
:1096B000164B1B68002BE9D05B68002BE6D020001E
:1096C0009847BB5900215B78122BDFD12000FFF7B0
:1096D00015FFDBE70E4BECE7112A04D1002900D07F
:1096E00032252900F2E7002D08D12000FFF732F9DA
:1096F000002803D0102302791343037121002800AE
:10970000FDF798FAC2E7C046F865FF1FF065FF1F36
:10971000F465FF1F70B50E4E8500AB590400002B99
:1097200013D01B78002B11D10A4B1B68002B04D0DF
:109730005B68002B01D02000984773595B78122B8F
:1097400003D100212000FFF7D9FE70BD024BECE7EA
:10975000F865FF1FF465FF1FF065FF1F094B8000D0
:10976000C3581020002B0CD01A6A002A09D09B681D
:10977000002B06D0127A1B7E101C9A4200D9181CAE
:10978000C0B27047F865FF1F70B503000D001400EC
:109790000220002A30D000292ED013700B78081D2B
:1097A00053704B789370FFF7A7FCE0700120022103
:1097B0002B7A23716B7B034063716A7B0A401343EE
:1097C000042263716E7B1640334363716E7BF6082F
:1097D000F600334363712B7B0340A371287B014068
:1097E00000200B43A371297B0A401343A3712A7BFA
:1097F000D208D2001343A37170BD10B50A00010056
:109800000120FFF7C1FF10BD10B50A0001000220C2
:10981000FFF7BAFF10BD70B506000C000220002E45
:1098200030D000292ED07378201D0B70B3784B7088
:10983000F178FFF76DFC01223579257271794B10B3
:1098400008001340934010400343881010408000EC
:10985000C9080343C9000B436373B1794B10080077
:109860001340934010400343881002409200C908FF
:109870001343C9000B4321202373FCF773FE854279
:1098800001D2122070BD2220257AFCF76BFE8542A2
:10989000F7D823781820042BF4D86378012BF1D85B
:1098A0000020EFE7030010B50220002909D0002BAB
:1098B00007D00322481C0A7019000D3202F098F8F4
:1098C000002010BD03000222080010B5002B06D0B6
:1098D000002904D00E32591C02F08AF80022100030
:1098E00010BD030010B50220002909D0002B07D0BD
:1098F0000422481C0A7019000C3202F079F800208A
:1099000010BD10B5FFF7DEFF10BD030002200029D7
:1099100006D0002B04D0052200200A701B784B7063
:10992000704703000220002B08D0002906D05B7886
:1099300000200B70013B082B00D918307047030042
:1099400010B50220002909D0002B07D00622481CA0
:109950000A7019000A3202F04BF8002010BD10B551
:10996000FFF7B0FF10BD02000B00022010B5002968
:109970000ED0002A0CD00721197011885970118857
:10998000090A997011180822D81C02F031F8002039
:1099900010BD03000A00022010B5002B0CD00029D6
:1099A0000AD099785878090201431180901CD91C7B
:1099B000082202F01DF8002010BD030010B502209F
:1099C000002909D0002B07D00822481C0A70190072
:1099D000921802F00DF8002010BD02000B000220CA
:1099E00010B500290BD0002A09D00921197011786F
:1099F00018185970511C062201F0FAFF002010BD02
:109A000010B5FFF75FFF10BD02000B00022010B57C
:109A1000002A09D0002907D05178197011180622A0
:109A2000581C01F0E5FF002010BD030010B5022016
:109A3000002909D0002B07D00A22481C0A701900FF
:109A4000063201F0D5FF002010BD10B5FFF73AFF38
:109A500010BD02000B00022010B5002A06D000291C
:109A600004D018005178FFF753FB002010BDF0B56B
:109A700085B017001E006A46062305000800918184
:109A80009380FEF7C0FC1324011E02900CD0380016
:109A9000B047041E05D1280001A9FEF76FFA041E85
:109AA00002D0029801F0E4FE2800FFF701FA20003E
:109AB00005B0F0BDF0B504008BB001911500002198
:109AC000102202A802F034F8334EA700B85900283B
:109AD0003CD0C388A34239D10378002B36D14278D9
:109AE000062A18D102000100553235310C3006AB80
:109AF000FFF7A9FA002829D12000FFF72FFE020066
:109B000006A902A801F074FF200002A901F0D8FE06
:109B100001200BB0F0BD816E002917D00B8A112AED
:109B200028D19D420ED101981231093A01F020FF4F
:109B3000012807D1BB5920009D6EFFF70FFE2900B9
:109B40000200DEE732212000FFF7D8FC2000FEF7FC
:109B500001FF061E1BD0416A002918D00B8AAB42B8
:109B600015D108220198123101F002FF01280ED10F
:109B7000716A0AE09D42E9D108220198123101F090
:109B8000F7FE0128E2D1BB59996E8A7EB9E7200021
:109B900001F0AEFEBCE7C046F865FF1FF0B56B4DA7
:109BA00087007E5985B0337802900393002B00D054
:109BB00087E0B368346A01937078062817D10122D0
:109BC0001B7D134202D0217B114218D10222134285
:109BD00002D0217B114251D10422134203D0237BB6
:109BE000134200D08BE0019B5A7DEB5991E007387E
:109BF0000428F8D801F0ACFE032E42678300B36E50
:109C0000002B03D11C2001F063FEB066EB599C6E63
:109C1000002C1CD010220021200001F089FF0298A6
:109C2000FFF79CFD01002000FFF72DFA01F0F8FC82
:109C30002082200008211230FFF725FA0298FFF752
:109C40008DFDA076EB592100D888FFF70FFC082284
:109C5000EB591CE0B36E002B05D01A00198AF0886E
:109C60001232FFF70DFC0222019B197DEB591142C4
:109C70003DD0207B10423AD0073208E0F488FCF750
:109C8000DBFD01002000FFF711FC0A22EB595A709E
:109C9000029B9C002A595378073B042B11D8D0888B
:109CA000FEF758FE00284ED0C3895A08D21828491A
:109CB000029B0298CB542B5941180433254801F0DC
:109CC0006FFD05B0F0BDFCF79FFD0300012083424E
:109CD00001D100200393EB59DE88FCF79BFD03992B
:109CE00002003000FFF7ECFB019AEB59117D0422D2
:109CF00011420CD0217B114209D00B22C7E7F68814
:109D0000FCF73CFD01003000FFF7EEFB6BE7019A2A
:109D1000527D01210A4204D0607B084201D00C220E
:109D2000B5E702210A4204D0607B084201D00E222E
:109D3000ADE704210A4204D0627B0A4201D010221E
:109D4000A5E71222A3E7FA225200B0E7F865FF1F49
:109D5000FC65FF1F13A1001110B5064B1A780423F0
:109D6000100018401A4200D00348FFF727FA0020DD
:109D700010BDC0468564FF1F4043FF1F70B504003F
:109D8000FFF7D4FA051E43D12000FFF77FFA234ED8
:109D9000A400A0598268937CDB0708D50321036ADD
:109DA0001B790B40012B02D1017F0B430377431D2D
:109DB000D97F8B1E022B0DD8022900D00121C0882B
:109DC000FCF790FF042133591A7F59700A431A7720
:109DD000280070BD01290CD10223102243700021FC
:109DE0000C3001F0A5FE305910213530FFF74BF94A
:109DF000EEE70529ECD10223D118437010220C3074
:109E000001F0F6FD04233259117F0B431377EAE783
:109E100008251828DCD1053DDAE7C046F865FF1FA4
:109E2000F0B58BB0059143887E4F9E00F459150024
:109E30000493002C15D1012902D000200BB0F0BDF5
:109E4000101D57781678FFF757F9EB683200029328
:109E50002B7A0499019300903B002000FCF70CFF43
:109E6000EBE7E388049A934201D00820E6E72378E1
:109E7000012B00D1D4E0059B581E092800D9CFE062
:109E800001F066FD05CE0A29CC506C859AB22900F6
:109E90000498FFF773FFD1E7200029001022453016
:109EA00001F0A6FDB9594B78042B02D1013B4B7050
:109EB000C3E70B000A00253335320C310498FFF755
:109EC00095F90498FFF702FA0522431E9841BB5901
:109ED000C0005A70B2E7200029001022553001F06E
:109EE00087FD049B4F4C9D00295904980A0006AB3E
:109EF00055320C31FFF77AF929591022453106A85D
:109F000001F036FD012808D10498FFF7F7F9059014
:109F1000002804D106222B595A7005988EE7082391
:109F20000593FAE763780C2B7AD1E36E002B03D10B
:109F30001C2001F0CDFCE066BB59D86E00286FD024
:109F40001022290001F054FDBB590498DC6EFFF784
:109F500005FC0D22A076BB595A706EE7E06E002812
:109F60005ED063780D2B5BD12B8808220382A91C5D
:109F7000123001F03DFDBB599A68517D0222114219
:109F800026D0186A407B104222D00C32E4E7637876
:109F90000E2B45D1236F002B03D1162001F098FC26
:109FA0002067BB59186F002803D01022290001F048
:109FB0001FFD0F22BB59CFE763780F2B30D1206FE5
:109FC0000622691C103001F013FDBB599A68517DBF
:109FD0000422114203D0196A497B1142D5D10021D4
:109FE0000498FFF78BFA28E7636F002B0DD0BB595D
:109FF000586F0028F3D01022290001F0F9FC01224B
:10A00000BB5952425B6F1A61E9E7142001F060FC12
:10A01000BB5960675B6F002BE9D126E72978DFE742
:10A0200007200BE7F865FF1F10B5064C207001F004
:10A0300047FD06212078FDF791FF0348FEF778FCE5
:10A0400010BDC0460B66FF1FC991001100200BB266
:10A0500070B50D00834216DA264B187801F050FBDC
:10A06000041E0DD00378922B0ED0A02B37D0224B9C
:10A070001878FF283AD0210001F0C2FA002835D123
:10A0800080200002684070BD43780E2B0BD03E2B21
:10A09000EDD18378052B12D0082BE8D18179808807
:10A0A000FFF7D8FA08E0154B82889A42DFD183681F
:10A0B0001878591CFEF7C0FE002817D1D7E7104BBF
:10A0C0001B785B0712D50F4B1B68002B0ED09B68CB
:10A0D000002B0BD0C289811D80889847ECE7FFF7E1
:10A0E00041FAA068002801D001F0C2FB200001F075
:10A0F00047FDC5E70B66FF1F3943FF1F182000000F
:10A100008564FF1FF465FF1F10B50078FFF712FA92
:10A1100010BD10B50078FFF7FDFA10BD0C234343C6
:10A12000084A10B59B185A68002A03D0012901D1AA
:10A13000904710BD9B68002BFBD00029F9D19847B0
:10A14000F7E7C0462866FF1F01238340094A10B580
:10A15000946B1C439463506B98435063D46B200002
:10A160009843012901D120001843D063116B0B43A0
:10A17000136310BD00800040F0B500240127154B8B
:10A1800085B0DA6B144E03921A6C0192DA64019B6B
:10A19000E3403B4217D0039DE5403D400295E5B2C8
:10A1A00002992800FFF7BAFF316A736A002908D0C4
:10A1B0003900002B01D0029979402800FFF7C4FF35
:10A1C00001E0002BF9D101340C36172CDFD105B09A
:10A1D000F0BDC046008000400C66FF1F064B012109
:10A1E0005A68C2400A4204D01B68C34018000840A5
:10A1F00070471B6DF9E7C046008000400122064B06
:10A200008240002903D0D9680A43DA607047D968D0
:10A210009143D960FAE7C0460038004030B50324C6
:10A2200044430F4BE25C1B199C785D7801232D1B86
:10A230000135AB40013BA340A140DB430C00122899
:10A2400007D808499200521811681940214311603B
:10A2500030BD054A11680B4023431360F8E7C04640
:10A26000B3BE001108F0004014F00040C21F70B5EA
:10A27000D4B20623092C0BD80125084C954000299F
:10A2800008D00021FFF7CAFF23682B432360002377
:10A29000180070BD2368AB43F8E7C04600380040A3
:10A2A000214BF0B51B185B78022B21D103244443CA
:10A2B0001E4A1F4EA35C1219947801221500854096
:10A2C000B76B013CE4B23D43A240B563194C122880
:10A2D00015D89B0000290CD117495B1899680A43CF
:10A2E0009A600123205C154A834011680B43136078
:10A2F000F0BD11495B18996891439960F1E70E4BE5
:10A3000000290DD159690A435A61225C1328E8D00B
:10A310000123203A93400A49086803430B60E7E7AA
:10A32000596991435961F0E70C66FF1FB3BE0011F4
:10A3300000800040F8BE001100F00040A0F0004096
:10A34000A4F00040F8B500241B4E1C4D1C4B1B5DB7
:10A35000012B1FD1194A9269E2401A420BD0012207
:10A36000B25693402200143AD2B2022A09D81549B3
:10A370004A6913434B61013402360C35172CE5D181
:10A38000F8BD0022B2560F499200521891680B4353
:10A390009360F0E7022BEED1E7B23800FFF71EFF23
:10A3A00001235840C1B23800FFF77AFF3800FFF7A9
:10A3B00015FF6877DFE7C04685BE00110C66FF1FFA
:10A3C0000D66FF1F00F00040012202388240054B5D
:10A3D000002903D059690A435A617047596991436A
:10A3E0005961FAE700380040F8B50E0001210F006E
:10A3F0008740114A0400D368FD43BB43D360831EEA
:10A400008B4201D8FFF7E0FF00212000FFF72EFF6D
:10A410000A4A0B4B5168012E05D139431B19516073
:10A420005E700020F8BD2940516002221C19627044
:10A430009A6915409D61F4E70038004000800040B3
:10A440000C66FF1F012210B58240074B002906D081
:10A4500019680A431A600121FFF7C6FF10BD196889
:10A4600091431960F7E7C046008000400C2370B5A7
:10A47000002543430A4A29009B181D70094B04001C
:10A480001B185D70FFF7B0FF0123A34006492800A9
:10A490000A681A430A6005490A689A430A6070BD4F
:10A4A0002866FF1F0C66FF1F34800040308000408C
:10A4B00070B504000E00FF2813D003250540FFF7F8
:10A4C000D5FF084AA3089B009B183F22ED00AA4035
:10A4D000AE40196820009143314319600121FFF714
:10A4E0008DFE70BD18380040F8B50C244443134B62
:10A4F0000500E4186368002B03D1A3681220002B29
:10A500001AD0022201270E4B00215B195A70280035
:10A510002770FFF769FF63681E1E08D0A3683E001E
:10A52000002B04D02800FFF759FE4640F6B2280061
:10A530003100FFF709FE0020F8BDC0462866FF1F66
:10A540000C66FF1FF7B5C420FF222B4B8000195863
:10A55000002491433F3A0A431A508022274F520267
:10A56000274E1A60274B1D5D002D21D0A31E012B05
:10A5700003D80121E0B2FFF727FF012D18D11F4BAF
:10A580009B69E3402B4213D0E3B218000193FFF71D
:10A5900025FE01000198FFF755FFE3B2143B022BA3
:10A5A0001DD801217156184A8D405369AB43536140
:10A5B0003B7F002B0DD0E5B22800FFF795FF280068
:10A5C000FFF70CFE7B7F0100834202D02800FFF7DB
:10A5D000A5FD01340C370236172CC3D1F7BD01217C
:10A5E00000237156F3568D40074A9B009B189A68CA
:10A5F000AA439A60DCE7C04600E100E00C66FF1F5A
:10A6000085BE00110D66FF1F00F0004070B50E0002
:10A6100015000400FFF72AFF0C236343094A2000BA
:10A620009B189D605E60FFF75FFFF021064B074AB5
:10A630008900051E5A5002D02000FFF717FF28009E
:10A6400070BDC0462866FF1F0000FF1F79A10011E2
:10A6500070B5134D07202C78002C1FD198222100B3
:10A660005200280001F07CFA0123C420FF222B7045
:10A670000C4B80001C635C630B4B1C605C600B4BE1
:10A68000195891433F3A0A431A50802252021A60E5
:10A690000D20074A074901F09BF9200070BDC04614
:10A6A0000C66FF1F00800040A0F0004000E100E0C9
:10A6B00045A5001145A30011030010B50620072B86
:10A6C00009D8054A137001F00BFAD7210020034B7B
:10A6D000034A89005A5010BD6843FF1F0000FF1F46
:10A6E000D91AFF1F70B51D0002240C2910D8094A81
:10A6F000CA40D2070CD5FBF741FF041E08D1059ACA
:10A7000004992800FBF756FFFCF7C4FDFFF724FB74
:10A71000200070BD1210000030B50D7802232C000F
:10A720009C43184201D02B431C0008252300AB4357
:10A73000284201D02B00234320241D00A5432042A2
:10A7400001D01C4325002A230D70184204D0117833
:10A750001E3B0B43137030BD0028FCD10C21137835
:10A760008B43F7E7F8B51D0006AB1B88140007AA5A
:10A770000E000B201778002B27D10A78022A49D126
:10A780004A68507811780002244A08438018042847
:10A7900040D801F0DDF803121D1B2300F06800F023
:10A7A000B7FF021CC0B2B84200D93A1CD2B2200096
:10A7B000F1682A8001F01CF906E00222F3681B8888
:10A7C0002A8023701B0A63700020F8BD0622EEE782
:10A7D00001232B80F3681B782370F5E7F368002BC7
:10A7E00016D008222A801A8822701A88120A6270EB
:10A7F0005A88A2705A88120AE2709A8822719A883E
:10A80000120A6271DA88A271DB881B0AE371DBE746
:10A810002B80D9E701202B80D7E7C04600D6FFFF69
:10A82000F7B516000A781D0008AB1F880C0001233D
:10A83000022A18D14A685078117800022B4A08433E
:10A84000801803280FD801F083F802254439E06806
:10A8500000F05EFFC0B20723B84204D37B19019316
:10A86000152B02DD0D231800FEBDE0682A00310023
:10A87000C01901F0BDF86B4600209B88E268D054F7
:10A880001B4B1B68834203D01B68834200D0984750
:10A890000023E8E70B23002FE5D1022DE2D17378E6
:10A8A00032781B021343E2681380114B1B68002BA4
:10A8B000EED01B68002BEBD00120E8E70B23002F24
:10A8C000D1D1062DCED12A003100E06801F090F8F8
:10A8D000DEE70B23002FC6D1012DC3D132787533AB
:10A8E000012AC0D8E3681A70D2E7C04600D6FFFF3D
:10A8F0001868FF1F70B50C001500072837D801F045
:10A9000027F8041436361B36242E182015290BD8A8
:10A91000184E16220021300001F00AF92200290009
:10A92000300001F065F8002070BD18200229FBD12D
:10A930001288114B1A80F6E718200829F4D10A0072
:10A940000E48290000F0ACFFEDE718200129EBD1FB
:10A950000B4B10780B49DA69FFF7DEFEE3E71820AE
:10A960000129E1D1064B10780749DA6BF4E70220A0
:10A97000DAE7C0460068FF1FE643FF1FDC43FF1F06
:10A980006C43FF1F9443FF1FB443FF1F030010B528
:10A990000020DB0704D50721024A034800F08CF8A9
:10A9A00010BDC04610BF00116C43FF1F054A0300D5
:10A9B0001068002803D082889A4201D180687047CD
:10A9C0000068F6E7106AFF1F0A88030008009A4231
:10A9D00004D08A8804309A4200D0002070470000DA
:10A9E000F8B5F22200230D4F0D4E79680500424361
:10A9F0003370994200D07B600A4C0021200001F0A6
:10AA000097F800231A007C60AB4202D1002033701B
:10AA1000F8BD01332280DBB2F234F5E7086BFF1F8B
:10AA2000066BFF1F146AFF1F73B56B46019006008B
:10AA3000684615001980FCF75FFF041E11D1002D38
:10AA40000FD07689002E11D00C2000F041FF002895
:10AA50000ED0084A0460136886808560002B02D1FE
:10AA60001060200076BD1A001B68F7E70224F8E7A3
:10AA70001324F6E7106AFF1F012100220A4B10B5CC
:10AA800049420A4C198099809A719A70084B20703B
:10AA9000012019805A60FFF7A3FF2078FCF78AFF96
:10AAA0000448FDF745FF10BD2068FF1F106BFF1F16
:10AAB000086BFF1F65AB0011022310B5002802D000
:10AAC000FFF7B2FF0300180010BD0000030010B52F
:10AAD0000020DB0704D50421024A0348FFF7A4FF46
:10AAE00010BDC04624BF0011EC43FF1FF0B50E2679
:10AAF00087B003930CAB1F8802ABF6180500080063
:10AB000031000292FDF77AF804000120002C0FD0EA
:10AB10003088FFF74BFF03000E20002B08D05E6843
:10AB2000002E05D021002800039B029A0097B04711
:10AB300007B0F0BD0A4B10B5984207D1012200239F
:10AB400052420A808B708A808B7110BDFFF73CFFE8
:10AB50000028FAD001235B42038000238370F4E7CE
:10AB6000FFFF0000F8B5050001290AD1134E0024AB
:10AB70003388F227AB4219D028001149FFF7DAFFDA
:10AB800006E0022904D10139FDF750FF0028EDD07D
:10AB9000F8BD3B0063437268D018D35A002B09D02C
:10ABA0003A00002100F0C4FF0134E4B2054B1B78E9
:10ABB000A342EED801235B423380DDE7086BFF1F21
:10ABC0002068FF1F066BFF1F10B5FFF7FDFE030097
:10ABD0000020834200D0987810BD0000F0B589B005
:10ABE0001C000EAB80CB03901E8810AB1B78049228
:10ABF00002930B7A0D00DB0616D42B780593022BFB
:10AC000024D00498FFF7D2FE002812D003689C4697
:10AC1000002B0ED0029B2200019329003B006446CA
:10AC200003980096A04705E00498FFF7BFFE0028B0
:10AC300002D10E2009B0F0BD8368002BF9D00A22A2
:10AC40002900039898470028D7D0F3E76B68587815
:10AC50001A786B4B000210439842D2D8043B9842BA
:10AC600010D2684B984242D015D8674BC0180128C3
:10AC7000C7D80B20002EDDD1EB681A7859683A80CE
:10AC8000200028E0614BC018032800D979E000F0CB
:10AC90005FFE846A789E5E4B9842B2D10B20002EF4
:10ACA000C8D101233B80EB6831001B782370688991
:10ACB000013080B2FCF7A2FF3A88031E0ED0017863
:10ACC00002328A183A80428962704289120AA2705E
:10ACD00059680278E01C00F08BFE06E004323A80EE
:10ACE00031000422601C00F023FF0020A2E70B20AB
:10ACF000002E9FD1EB6807A91E8804233B80330AEE
:10AD0000300026706370FCF779FF051E28D004AB75
:10AD10009A890E2304A95B183E49C668FCF7E2FF36
:10AD200000280BD12B783C486A680599FBF798FB03
:10AD3000002803D1012304AA5B42D3813278022A7E
:10AD400006D17168201D00F053FE3B8802333B8022
:10AD50000E2304AA9B181B88A3701B0AE370C4E788
:10AD600004ABDE81F4E70B20002E00D062E7E96837
:10AD70000398FFF729FF02233B802070000A6070D0
:10AD8000B3E70B20002E00D054E70222EB681B88AB
:10AD90003A8023701B0A6370A7E7E86800F0B8FCEC
:10ADA000C2B203000720B24200D243E70DD002999D
:10ADB000DBB27118994202DB921BD3B20293029B61
:10ADC000E9681A003B8089195AE70023F6E70B204F
:10ADD000002E00D02EE70722EB683A801A78227006
:10ADE0005A7862705A88A2705A88120AE2701A79E8
:10ADF0002271DA886271DB881B0AA37175E7C0468D
:10AE0000042900000228000000D8FFFFFFD6FFFF42
:10AE100003280000FFFF000054BE0011F0B58DB004
:10AE20006B460020089120229B5E83423DDAA64BB0
:10AE3000187800F065FC071E32D00378B02B2CD1B7
:10AE40000079023816281FD800F0E2FC17001E0017
:10AE50001E001E0031001E0096001E001D011E0077
:10AE600052011E0073011E00CD011E0050021E0083
:10AE70001E001E008E021E00E302944B94491B88A4
:10AE800078880B80FBF72CF83800FCF7ADFF914B6E
:10AE90001B68002B01D038009847380000F070FE86
:10AEA0008020089B0002434018000DB0F0BDEE2248
:10AEB0000021874800F03CFE0BAA3B7B798938894A
:10AEC00000923A000D32FCF7B1FD0400804B1B7874
:10AED000002C3FD146E0804B788805937F4B4100A2
:10AEE000CB5A0BAE073BDBB23288029300230193AF
:10AEF0007B4B210006930093059BFFF76FFE744D7B
:10AF0000002810D1069B3A8A1B889A420BD1380040
:10AF10000599123000F02CFD002804D02B786289AE
:10AF20009B00EB185A80162306A81B1832882000B5
:10AF30007989FCF7D7FE2B7804009A00AA1851886B
:10AF40000029C3D00133DBB22B70002807D006A93B
:10AF5000C98A9180634A12889A42BCD802E00121D2
:10AF600049429180002B04D059497888FAF7ECFFC8
:10AF70008AE73E890A2479E000253E89574B0693EB
:10AF80007B88069A5B009B5A033B9D4202DB002DA7
:10AF9000F0D05BE0162206A812183B7B798900925C
:10AFA0003A0030000D32FCF741FD0590002858D0E2
:10AFB0004689017A7888FCF703FD041E44D1464B8C
:10AFC00078880793069B4100C95A454B0439C9B29A
:10AFD00006AAD28A06930291019400930599079BD1
:10AFE000FFF7FCFD041E2FD1069B39491A88931CDC
:10AFF000002D26D14B807988384B4900CB5A511906
:10B00000033B8B4220DD059B31485B8941190B7165
:10B01000A91C0135C9B2EDB2059145191B0A2B7166
:10B02000059B2D490433181800F0E2FC2C4B059ABF
:10B030001B88D318DDB22C4B9E4205D00136B6B228
:10B040009CE749889942D6D0002D0CD0204C28008E
:10B05000618800F0F5FA207021007888FAF784FF03
:10B0600012E7059CF0E7002C00D183E77B78142BD6
:10B0700000D109E716493B794E800B700C71788836
:10B08000FAF724FF00E7162406ABE41821003889FC
:10B09000FCF7B4FD011E00D1B7E1788822880F4C7F
:10B0A00045002C5B0A4D013CE4B2029400240F4B96
:10B0B00001940095FFF792FD041E00D014E12900D1
:10B0C0007888FAF761FFDFE6106BFF1FD842FF1F99
:10B0D0002868FF1F1C68FF1F1C69FF1F5864FF1FA3
:10B0E0000C6AFF1FD642FF1FFFFF00002A68FF1FE8
:10B0F000162406ABE41821003889FCF77FFD011EF9
:10B1000000D182E178882288AE4C45002C5BAE4DA0
:10B11000013CE4B202947C89AC4B01940095FFF7AA
:10B120005DFD041E00D0DFE029007888FAF736FFC5
:10B13000AAE60025A44B1D803B00F6331B78A24AEB
:10B1400078880792AB4208D99E4B128806930699DD
:10B1500043005B5A013B9A4203DB0799FAF728FF49
:10B1600092E616246B00FB18059306ABE418059BCA
:10B1700021001889FCF742FD011E03D1059B012423
:10B180001E8973E77888924B2288069C09934300B6
:10B190001B5B904E013BDBB20293002300960193B0
:10B1A000099BFFF71BFD041E02D0059B1E895DE76E
:10B1B0007B88069A5B009B5A079A1088328812187F
:10B1C000934202DC1B1A013B33807F4C02303288F1
:10B1D0000999001900F00CFC2388328801359B186E
:10B1E0002380EDB2A8E70BAA3B7B798938890092CE
:10B1F0003A000D32FCF71AFC00250590059B002B48
:10B2000004D10A24002D00D16EE060E0059B78880F
:10B21000197AFCF7D5FB0100041E63D1694C6C4B15
:10B22000788806940993069B4400E45A694B063CCF
:10B23000E4B20BAE32880793029401910093059912
:10B24000099BFFF7CBFC041E4CD1079B5E491B8872
:10B250001A1D002D30D14A80059B5B4C5A89631919
:10B260001A716B1C9BB2E318120A1A71162306A8F6
:10B2700032881B1879890598FCF734FDFF21AA1C38
:10B280002E1D03350B00059092B2B6B2ADB2002868
:10B2900003D006ABDB8AD9B21B0AA218651911715B
:10B2A0002B714C4D301D2A884949201800F0A0FB15
:10B2B0002B88F618B5B2A1E74988914207D17A8860
:10B2C00006995200525AEB18053A9A42C4DC3E4C99
:10B2D0002800618800F0ACF9207021007888FAF726
:10B2E00071FED1E5002DF2D13E89BFE6162606ABF0
:10B2F000F61831003889FCF781FC3D000400FA356E
:10B3000000282DD0037A9B060CD400227B89398932
:10B31000788800923A000C32FFF7E8FB041E10D048
:10B320003E8915E03088FFF741FB00281AD083687A
:10B33000002B17D02100122278889847041EE4D0F1
:10B34000EEE72B78002B02D17888FAF74BFE002627
:10B350002B78002B00D097E5002C00D194E585E6F2
:10B360000124DDE70E24DBE7162506ABED182900E6
:10B370003889FCF743FC041E47D0037A9B0611D49E
:10B38000154A7B881188994203D01448814207D11D
:10B390001380134BF2261D780023D9B2A94221D382
:10B3A0000924A1E72888FFF701FB00282FD0836834
:10B3B000002B2CD02100122278889847041EDFD061
:10B3C00092E7C0465864FF1F2868FF1F2A68FF1FC6
:10B3D0001C69FF1F0C6AFF1F086BFF1FFFFF0000A7
:10B3E000066BFF1F31005943546801336018615ADE
:10B3F0000029D2D13C0008342100F22200F0F8FAF2
:10B4000021007888FAF7F6FD3EE501246CE70E246A
:10B410006AE71D4B1A887B889A4231D07888FAF700
:10B42000F3FD31E5F223059851684343CD18C95A1D
:10B4300000291FD03B7A012B0BD16C88AB88788810
:10B44000AA1D0094FFF752FB041E02D000233B729A
:10B450002E88F2220021280000F06AFB00232B80B6
:10B46000059B0133DBB20593084B05991B78064A0F
:10B470008B42D7D801235B421380002CCED0F5E558
:10B48000002634000596EFE7086BFF1F066BFF1FD1
:10B4900070B504000E001500FFF796FA031E08D1E0
:10B4A00031000548FFF790FA03001120002B02D06D
:10B4B0001C8000209D7070BDFFFF0000F8B50B4F91
:10B4C00006003B780D001400FF2B0ED00A2000F080
:10B4D000D7F9011E09D0B1230380002346800371F0
:10B4E000C5800481387800F08BF8F8BD2D44FF1F2B
:10B4F000F7B50F0008A90600088809A90B240988D8
:10B50000002821D10234022B1ED1557813782D0248
:10B510001D432B008B4301937334002B14D1FB6824
:10B52000300019000093FFF74FFB019C85420BD0C0
:10B530002A0030000099FFF7ABFF041E04D12A0057
:10B5400030007989FFF7BAFF2000FEBDF0B50E7814
:10B5500085B003900AA805880120022E0DD14C6801
:10B560002778647824023C43054FBC4205D10398F8
:10B57000DBB201960095FFF7BBFF05B0F0BDC046FA
:10B5800002290000034B10B51B68002B00D0984720
:10B59000FEE7C046146BFF1F07B501A8FFF7F2FFD7
:10B5A000044A05480021121A00F0DAFAF8F722F9E5
:10B5B000FEE7C046186BFF1F3044FF1F000000006D
:10B5C00001B40248844601BC604700BF456B0100DE
:10B5D00001B40248844601BC604700BFD92FFF1F59
:10B5E00001B40248844601BC604700BFB14E000070
:10B5F00001B40248844601BC604700BF45510100C8
:10B6000001B40248844601BC604700BF594F0100A5
:10B6100001B40248844601BC604700BF1930FF1FD7
:10B6200001B40248844601BC604700BF29510100B3
:10B6300001B40248844601BC604700BF090E000007
:10B6400001B40248844601BC604700BF350E0000CB
:10B6500001B40248844601BC604700BFC9A900008C
:10B6600001B40248844601BC604700BF014C0100A0
:10B6700001B40248844601BC604700BF791800004D
:10B6800001B40248844601BC604700BF01240000A9
:10B6900001B40248844601BC604700BF7D18FF1F0B
:10B6A00001B40248844601BC604700BF5D1700003A
:10B6B00001B40248844601BC604700BFADAE000043
:10B6C00001B40248844601BC604700BF792DFF1FCA
:10B6D00001B40248844601BC604700BF055E00001B
:10B6E00001B40248844601BC604700BF55220000F7
:10B6F00001B40248844601BC604700BF193AFF1FED
:10B7000001B40248844601BC604700BFF54E010009
:10B7100001B40248844601BC604700BFDD5201000D
:10B7200001B40248844601BC604700BF8B5201004F
:10B7300001B40248844601BC604700BFA54F010028
:10B7400001B40248844601BC604700BF4D1F0000A1
:10B7500001B40248844601BC604700BFE117000005
:10B7600001B40248844601BC604700BF4D38FF1F4A
:10B7700001B40248844601BC604700BF2932FF1F64
:10B7800001B40248844601BC604700BFC52DFF1FBD
:10B7900001B40248844601BC604700BF75A900009F
:10B7A00001B40248844601BC604700BFA9460100BD
:10B7B00001B40248844601BC604700BF1147010044
:10B7C00001B40248844601BC604700BFD91B000099
:10B7D00001B40248844601BC604700BF51470100E4
:10B7E00001B40248844601BC604700BF0132FF1F1C
:10B7F00001B40248844601BC604700BF9136FF1F78
:10B8000001B40248844601BC604700BFEDA50000BA
:10B8100001B40248844601BC604700BF413BFF1FA2
:10B8200001B40248844601BC604700BFB352010026
:10B8300001B40248844601BC604700BFF94C0100D6
:10B8400001B40248844601BC604700BF5952010060
:10B8500001B40248844601BC604700BFC135FF1FE8
:10B8600001B40248844601BC604700BF3555000062
:10B8700001B40248844601BC604700BFD9490100B9
:10B8800001B40248844601BC604700BF1D4D010061
:10B8900001B40248844601BC604700BFC51D0000DA
:10B8A00001B40248844601BC604700BF810E00001D
:10B8B00001B40248844601BC604700BF291C000057
:10B8C00001B40248844601BC604700BF311B000040
:10B8D00001B40248844601BC604700BF3D4B0100F3
:10B8E00001B40248844601BC604700BF851F0000C8
:10B8F00001B40248844601BC604700BF091B000038
:10B9000001B40248844601BC604700BF691F0000C3
:10B9100001B40248844601BC604700BF4537FF1FA1
:10B9200001B40248844601BC604700BF6571010054
:10B9300001B40248844601BC604700BF3938FF1F8C
:10B9400001B40248844601BC604700BFED39FF1FC7
:10B9500001B40248844601BC604700BF2D3BFF1F75
:10B9600001B40248844601BC604700BF350E0000A8
:10B9700001B40248844601BC604700BFCD4C0100C1
:10B9800001B40248844601BC604700BF5933FF1F21
:10B9900001B40248844601BC604700BF2146010053
:10B9A00001B40248844601BC604700BF4550000016
:10B9B00001B40248844601BC604700BFED4A010063
:10B9C00001B40248844601BC604700BFC12FFF1F7D
:10B9D00001B40248844601BC604700BF6130FF1FCC
:10B9E00001B40248844601BC604700BFC538FF1F50
:10B9F00001B40248844601BC604700BFE94C010025
:10BA000001B40248844601BC604700BFC56D010017
:10BA100001B40248844601BC604700BF25260000EF
:10BA200001B40248844601BC604700BF1D4B0100C1
:10BA300001B40248844601BC604700BF056A0000AB
:10BA400001B40248844601BC604700BFB54C010008
:10BA500001B40248844601BC604700BF8D1200005B
:10BA600001B40248844601BC604700BFE9280000D9
:10BA700001B40248844601BC604700BF6DBC0000B1
:10BA800001B40248844601BC604700BFC5210000E4
:10BA900001B40248844601BC604700BFF30E0000B9
:10BAA00001B40248844601BC604700BFC94A010096
:10BAB00001B40248844601BC604700BF9135FF1FB6
:10BAC00001B40248844601BC604700BFC92600009B
:10BAD00001B40248844601BC604700BF9DA9000034
:10BAE00001B40248844601BC604700BFD91AFF1F59
:10BAF00001B40248844601BC604700BFDD66010016
:10BB000001B40248844601BC604700BF8538FF1F6E
:10BB100001B40248844601BC604700BF9D35FF1F49
:10BB200001B40248844601BC604700BF7139FF1F61
:10BB300001B40248844601BC604700BF154D0100B6
:10BB400001B40248844601BC604700BF5118FF1F82
:10BB500001B40248844601BC604700BF017F000079
:10BB600001B40248844601BC604700BFB70E000024
:10BB700001B40248844601BC604700BF090E0000C2
:10BB800001B40248844601BC604700BF434D010038
:10BB900001B40248844601BC604700BF156B010038
:10BBA00001B40248844601BC604700BF0539FF1F4D
:10BBB00001B40248844601BC604700BF0D52010039
:10BBC00001B40248844601BC604700BF3D18000034
:10BBD00001B40248844601BC604700BF193BFF1F07
:10BBE00001B40248844601BC604700BF51250000F3
:10BBF00001B40248844601BC604700BFE54800002C
:10BC000001B40248844601BC604700BF8552010070
:10BC100001B40248844601BC604700BF21240000F3
:10BC200001B40248844601BC604700BF5549010089
:10BC300000030102020303030403050006020700D8
:10BC4000080209030A030B030C000D000E030F0387
:10BC5000100311031303140315021602BD3B001158
:10BC6000F13B0011000000000200000072BC001156
:10BC7000192A0F180A000000F1590000FD240000E5
:10BC800041460100398000114DA00011A17400113E
:10BC90003D7E0011195300111DAE0011814F00119E
:10BCA000CD3D0011FD3E0011000000001616000001
:10BCB00002000000BCBC0011F4FFF3FFD2FC000046
:10BCC0003D40001100000000000000005475796143
:10BCD0000042312E350030303137006769746875A5
:10BCE000622E636F6D2F7076767800544842310073
:10BCF0000200000004BD0011292A282A272A262A2A
:10BD0000252A242A0A180000E2040000710200001B
:10BD100078EC0000744000001027000060F0000084
:10BD200006640000204E0000000000000500000036
:10BD30001F501D00023CB400000117001500000058
:10BD4000A1020000303132333435363738394142C0
:10BD500043444546000000001D5700117157001173
:10BD6000000000000200000070BD00116F2A6E2A62
:10BD70001A18EAD8BC80F0FC600000000000000047
:10BD800000005F066B2F363D7D077F3F777C596E45
:10BD90007971000001A00000000000006410B71DD0
:10BDA000C8206E3BAC30D9269041DC76F4516B6BE9
:10BDB0005861B24D3C7105502083B8ED44930FF0AB
:10BDC000E8A3D6D68CB361CBB0C2649BD4D2D38661
:10BDD00078E20AA01CF2BDBDFB349B5F80000080AE
:10BDE0000010000000000000A36000112D7700117A
:10BDF000C7600011357B00114B6100110B7B0011F6
:10BE0000C1610011E17A001113620011A97C0011D7
:10BE10007B620011A97C0011AD620011637C0011EE
:10BE2000C1610011997A001139620011417C001141
:10BE300000000000000000001F630011417C0011A1
:10BE40008163001145770011052A042A012A002A7E
:10BE5000022903280128002801180018000000000A
:10BE60000000000000000000000000870101020146
:10BE700002010102010203030401030101010101A6
:10BE80000303020103000D000E0010001100130057
:10BE90001401070108010A010B011C011D02040223
:10BEA00005020702080219021A021C021D030103FF
:10BEB000020317000201000504000807000B0A0036
:10BEC0001716001D1C010201010504010E0D0111D0
:10BED00010011413011716011A19020201020B0AAC
:10BEE000020E0D02111002141302171603050403AB
:10BEF0000807030B0A030E0D0001020307090A0BD2
:10BF00000E0F101112141718191A1B1F20212200CE
:10BF100065A7001121A80011000000000200000028
:10BF20005ABE0011000000004DB5001100000000D5
:08BF30000200000058BE0011E0
:020000041FFFDC
:1000000000000000353D001178BC001174BC0011E7
:100010003C61FF1F00000000000000000000000025
:1000200000000000000000000000000000000000D0
:1000300000000000000000000000000000000000C0
:1000400000000000000000000000000000000000B0
:1000500000000000000000000000000000000000A0
:100060000000000000000000000000000000000090
:100070000000000000000000000000000000000080
:100080000000000000000000000000000000000070
:100090000000000000000000000000000000000060
:1000A0000000000000000000000000000000000050
:1000B0000000000000000000000000000000000040
:1000C0000000000000000000000000000000000030
:1000D0000000000000000000000000000000000020
:1000E0000000000000000000000000000000000010
:1000F0000000000000000000000000000000000000
:1001000000000000000000000000000000000000EF
:1001100000000000000000000000000000000000DF
:1001200000000000000000000000000000000000CF
:1001300000000000000000000000000000000000BF
:1001400000000000000000000000000000000000AF
:10015000000000000000000000000000000000009F
:10016000000000000000000000000000000000008F
:10017000000000000000000000000000000000007F
:10018000000000000000000000000000000000006F
:100190004D32FF1FAD30FF1FC1660100000000009F
:1001A000000000000000000000000000000000004F
:1001B000000000000000000000000000000000003F
:1001C000000000000000000000000000000000002F
:1001D000000000000000000000000000000000001F
:1001E000000000000000000000000000000000000F
:1001F00000000000000000000000000000000000FF
:1002000000000000000000000000000000000000EE
:1002100000000000000000000000000000000000DE
:1002200000000000000000000000000000000000CE
:1002300000000000000000000000000000000000BE
:1002400000000000000000000000000000000000AE
:10025000000000000000000000000000000000009E
:10026000000000000000000000000000000000008E
:10027000000000000000000000000000000000007E
:10028000000000000000000000000000000000006E
:10029000000000000000000000000000000000005E
:1002A000000000000000000000000000000000004E
:1002B000000000000000000000000000000000003E
:1002C000000000000000000000000000000000002E
:1002D000000000000000000000000000000000001E
:1002E000000000000000000000000000000000000E
:1002F00000000000000000000000000000000000FE
:1003000000000000000000000000000000000000ED
:1003100000000000000000000000000000000000DD
:1003200000000000000000000000000000000000CD
:1003300000000000000000000000000000000000BD
:1003400000000000000000000000000000000000AD
:10035000000000000000000000000000000000009D
:10036000000000000000000000000000000000008D
:1003700099B500110000000000000000000000001E
:10038000000000000000000000000000000000006D
:10039000000000000000000000000000000000005D
:1003A000000000000000000000000000591AFF1FBC
:1003B000000000000000000000000000000000003D
:1003C000000000000000000000000000000000002D
:1003D000000000000000000000000000000000001D
:1003E000000000000000000000000000000000000D
:1003F00000000000000000000000000000000000FD
:08183800206FFF1F4118FF1F84
:10184000024981F3088802F0EFFA0000206FFF1FC1
:1018500010B502F061FA072804D0122808D0022837
:1018600008D010BD044A0420136B01331363F8E75A
:101870000220F6E71420F4E70065FF1FF8B5070023
:101880000C0026002500503630785135002804D150
:101890000300287058342370F8BD2978CA00481E08
:1018A0008141A3183800A25C5B68C9B2FFF7D0FF82
:1018B00000280DD12B78DA00A218013350602B706C
:1018C0003378044A013B3370136A01331362D8E75B
:1018D0000123DFE70065FF1F5C234343074910B581
:1018E000C9180B0058331B78012B05D1FFF7C6FF31
:1018F000034A936A0133936210BDC0463465FF1FEB
:101900000065FF1F10B502F02FF9064A01211300F0
:1019100010CB4942D967044B136002F0D5FA20007E
:1019200010BDC04600E100E01000100010B504003A
:1019300002F01AF9024B1C6002F0C6FA10BDC04654
:1019400000E100E0431E5A425341A022F0B5D2010B
:101950005B421340154D164A40019B182A18127E0F
:101960008BB00191002A1BD01A000832D46F0022DC
:10197000E6B206AFE4B294420EDC2818C369002B2D
:1019800008D0019902AA117106AA049202AA16733C
:1019900003A898470BB0F0BD1978B9540132EAE7B3
:1019A0001A7D1A7806AB01261A70E6E7C067FF1F9A
:1019B00000400040F0B5254B04004001C25C85B0FA
:1019C000002A2BD01A18117E002927D0917E0029D9
:1019D00024D01179022921D11689D788D168F51B25
:1019E000ADB22A1C102D00D9102292B2BE4217D1DE
:1019F0001818012303710023C269C38003819A422E
:101A000006D06846032103730171029301A8904731
:101A10000820002C00D0192001F0FEFA05B0F0BD1E
:101A2000013C65426C41A0256442ED012C40084D0B
:101A30001B186419074D0633013A92B2AA42EDD041
:101A40001888461C1E80085C2070F5E7C067FF1FE1
:101A500000400040FFFF00000F220E4B10B59868B9
:101A6000104002380A280BD802F060F80D0A0B0A61
:101A70000A110A0A0A0A060002210020FFF762FF83
:101A800010BD0121F9E70020FFF794FFF8E7DB6FB5
:101A9000F6E7C046004000400F220E4B10B5986894
:101AA000104002380A280BD802F040F80E0A0B0A40
:101AB0000A120A0A0A0A060002210120FFF742FF61
:101AC00010BD01210800F9E70120FFF773FFF7E7D8
:101AD000DB6FF5E70090004013B5334C2378072BFC
:101AE0003DD8324B1A78324B002A39D180221968FE
:101AF00052020A431A60252001F0C4FE20232D4A19
:101B000011680B43802113606B460422C9050868E5
:101B10000733104228D080210422C905C86810422A
:101B20002ED080212020C905CA688243CA601422B1
:101B30001A701A78002A2FD18021C905C86820326E
:101B40000243CA6014221A701A78002A28D11A4B4C
:101B50001A7D22785A601D221A705932DA6013BD3C
:101B60001A6816490A40C5E7086802430A60142249
:101B70001A701A78002ACED01A78013AD2B2F7E752
:101B8000C8680243CA6014221A7019784A1ED2B279
:101B90001A700029F9D1C4E71A78013AD2B2C7E71E
:101BA0001A78013AD2B2CEE76843FF1F3044FF1FD4
:101BB0003CF000406043FF1F00200040FFFFFEFF9D
:101BC000564B70B51B68012B03D1554A936D0133F9
:101BD000936502F0D1F9534B534A1860534B544C60
:101BE0001A600123534A1360534A13602378002B71
:101BF00006D006225149524802F03EF800232370D5
:101C0000504A514B10681B78C1B2002B0ED14F4C7B
:101C1000C0B223785BB2002B4FDB237824785BB211
:101C200064B21B0424021B191B1813600B1C5029DF
:101C30004ED95023464A47491078DBB2FF2202288A
:101C40004BD10868444C454D267890432A789642FB
:101C500054D9227824782E78023B5D10A31B6B4365
:101C60005201D31A10335B111843086001F0CCFF06
:101C7000031F012B45D83A4B1B78002B06D0394B5C
:101C80001B78002B02D0002002F0E6F9A122364B8F
:101C900092009978354B4A431B689B188322920027
:101CA0009B181B78033B012B03D8AF20400002F0A8
:101CB00073F801222E4BDA8270BD237824785BB250
:101CC00064B2FF33FF341B0424021B190138ABE755
:101CD000CAB2022AAED20223ACE70868254C264DD0
:101CE000267890432A78964208D9227824782D784D
:101CF000023B5B10641B63435201B2E72378DBB203
:101D0000B2E70228D5D11D4B1B78013B022B03D92A
:101D10001B4B1B78022BCCD16C20C8E79809FF1F06
:101D2000FC0FFF1F3864FF1FFF3F0000141003402B
:101D30003C64FF1F0C10034000100340D50BFF1F35
:101D40007211FF1FB40003408C09FF1F680AFF1FB8
:101D5000490AFF1F94000340460AFF1F470AFF1F5E
:101D6000F908FF1F2209FF1F300DFF1F3409FF1F55
:101D7000BC0BFF1F440AFF1F450AFF1F1C09FF1F62
:101D80002309FF1F10B502F0D7F80022014B1A807B
:101D900010BDC0463664FF1F10B502F0FDF8A1214A
:101DA000054A89009478054A61431268044B521829
:101DB000528C1A8010BDC046300DFF1F3409FF1F22
:101DC0003664FF1F10B50D4B0D4A9978A1239B0077
:101DD0004B431268D218531DD97F0A4B1B88994276
:101DE00009D2441C07D0C82805D0D2695B1A5A43CF
:101DF000054B5343C01802F06FF810BD300DFF1FA4
:101E00003409FF1F3664FF1F7102000070B5244DB6
:101E10002B68002B28D001F0FFFE2B68D8402B68E0
:101E20000400002B27D001F0B7FE2B68D8401D4BD3
:101E30001D4A9978A1239B004B431268D118D25CAC
:101E400091239B00002A20D0CA580132CA50174B58
:101E500017491B680868834214D3D23B181A012A19
:101E60001AD0144B186070BD01F0D6FE124B1968E1
:101E700001F082FFD3E701F08FFE0F4B196801F0EC
:101E80007BFFD4E70D495B18E8E7CA500C4B1B6891
:101E9000DB68E418201AE4E7F530FF30E1E7C046DC
:101EA0001C08FF1F300DFF1F3409FF1F9C09FF1F77
:101EB0003864FF1FA009FF1F1808FF1F2DFF3F00F8
:101EC0004064FF1F70B504000D00282916D10300DF
:101ED000A433C2881B889B1A0B4A9BB293420DD92C
:101EE00006006A3605223100653001F0B5FF002892
:101EF00004D13100200001F037FF70BD290020001F
:101F000001F0B2FEF9E7C046FE7F0000F8B505001B
:101F1000012001F061FE134CA36AA26A9342FBD137
:101F2000114E336002F060F8104903000860104859
:101F3000426894460F4A17680022BC4501D24268A5
:101F4000BA1A0D4802603268AD18A422E562606AD0
:101F5000520302436262094A1278002A01D00F3B01
:101F60000B60F8BD00F00040340AFF1FE408FF1FBB
:101F700028100040180AFF1F1C0AFF1F1C09FF1F22
:101F800070B580241025E405A3682B43A36002F0FC
:101F900023F8A368AB43A36070BD0000F7B516003B
:101FA00080221C001023D2050191916805000B438B
:101FB000936000225A4BD7301A6001F0FDFD9D233B
:101FC0002A002F009B00EB58CA3201210092FC37F7
:101FD000002B01D00021009A386801F08DFE290005
:101FE000009BCB311A784F4BD3351A604B780A7867
:101FF0001B0213438A7812041A43CB781B0613433F
:10200000494A1BBA13604B790A791B0213438A7938
:1020100012041A43CB7931001B061343434A1BBAFF
:1020200013606B782A781B021343AA7812041A43B0
:10203000EB781B0613433E4A1BBA1360019A330226
:1020400013433C4A13603C4B22001B1B9C46032954
:102050003DDCB3089A0013005142B21A032A46D15C
:10206000354AE018511A827840781204000202437F
:10207000E05C043302430A600022FF2B4BDDF022B8
:102080002E4B12011A600F222D4B1A602D4A136835
:10209000002BFCD00023224A27491360091B321D64
:1020A0000B191B68043A180A23706070180C1B0E79
:1020B000A070E3700434002AF2DC802210213B6817
:1020C000D20501333B6093688B439360F7BD634651
:1020D000D578981893782D061B042B43157804396E
:1020E0002B43557804322D022B430360AFE7022ABD
:1020F0000AD1114AE05C511AE218527812020243E6
:102100000A6004339BB2B7E7012AB5D10A4A521AD2
:10211000E15C1160F5E7084959180A600433ACE73F
:10212000000004403C0004403800044034000440F7
:10213000300004400C00044000010440040004404E
:102140001000044014000440F7B5150080221C0064
:102150001023D2050091916807000B439360002380
:10216000654AD730136001F027FD9D233E009B0098
:10217000F9583B00CA363200FC33002900D07FE01A
:10218000586801F0B9FD390032785C4BCB311A60E8
:102190004B780A781B0213438A78AC4612041A4320
:1021A000CB78281D1B061343554A1BBA13604B7985
:1021B0000A791B0213438A7912041A43CB791B064E
:1021C0001343504A1BBA13604B7A0A7A1B0213431B
:1021D0008A7A12041A43CB7A21001B0613434A4A17
:1021E0001BBA1360009A2B021343484A1360220063
:1021F000474B1B1B0093009BCE785B1801938B7899
:1022000036061B0433430E78043833434E780431CA
:1022100036023343019E33600328ECDC0321A80817
:10222000431C9B002940800003292BD13849E51825
:102230005E18A9786D78E35C09042D0229431943DF
:102240003160030008330021FF2B2DDD314B324973
:1022500019600F21314B1960012327490B60304B66
:1022600019680029FCD006211B680B40042B20D0E4
:1022700080220020D20593680A318B439360FEBD13
:1022800001217DE7022908D121495D18E11849782B
:10229000E35C090219432960D3E70129D3D11C4922
:1022A0005918E35C0B60CCE7194818180160043337
:1022B000CAE7002310490B606346002B0CDC3B008F
:1022C000FC335A68102101325A608022D20593688B
:1022D00001208B439360D2E7009B9B181B68190A6F
:1022E00013705170190C1B0ED37004235B42917054
:1022F0009C440432E0E7C046000004403C00044037
:102300003800044034000440300004400C00044015
:102310000001044004000440080F000010000440C5
:102320001400044070B5061E19D002225A4B9B7946
:102330009343012B13D1594B1A78FF2A0FD15A78A6
:10234000FF2A0CD19A78FF2A09D1DA78FF2A06D120
:102350001A79FF2A03D15B79FF2B00D199E0504B0A
:102360000C201A78012A08D000224E4D1A702978C4
:102370000B00093B042B01D8212070BD4B1F012B02
:10238000FAD9454CA37B042B00D982E0A279032A19
:1023900000D97EE09A1ED2B2012A02D860881F2896
:1023A00077D9002E56D0012E73D1A0880128E3D012
:1023B000002907D1581E032803D801F0B7FB1217D4
:1023C00015122E702978481E032811D80025364B87
:1023D0001D602823237501F01FFEA84227D0A58089
:1023E000CAE702212970EDE70421FBE70321F9E7A1
:1023F00007390129C0D82D490968C96A8906BBD5A2
:102400002B4908780028B7D1012A01D9002BB3D174
:1024100002230B708021274D2633890128782375EC
:1024200001F012FD80212878890101F015FC0123BB
:10243000A380214B1B78002B0AD0FA2280211F4B4E
:1024400092001B8809025A431A4B187801F0B4FD18
:10245000002092E701F088FB2B78A680073B012B38
:1024600003D917482E7001F077FD114B114C1A78E3
:10247000002A06D080210022207889011A7001F0FC
:10248000E3FC01F021FD80212078090201F0DCFC51
:10249000DEE7122071E7C046A60BFF1F6B09FF1F86
:1024A0001A09FF1F1C09FF1F4809FF1F4064FF1F77
:1024B0002309FF1F1B09FF1F2109FF1F2C09FF1FF5
:1024C0000010004010B5002901D001F04DFD10BDF5
:1024D000F7B5604B01919978A1239B004B435E4A6D
:1024E000060014681022E418D6235B00E058362357
:1024F000FF33E35C00279343222B41D1574B0F3A24
:102500001A600760012501F05FFC019B1880E82339
:102510005B00E35C002B01D0B34258DD0023504F39
:10252000FB70AD33FF33E3581A68002A03D09B8851
:10253000DB439B071DD03823FF33E35C002B18D00F
:102540009B235B00E35C002B13D1D133FF33E35CAF
:10255000B3420EDAA4235B00E15AE018090A023103
:1025600001F0F2FB23000122FE33013E01351A8700
:10257000FA70E8235B00E35C002B2AD0A8B2FEBD12
:1025800003683D00002BBED081880430090A023167
:1025900001F0DAFBD6235B00E3581F60B2E72300AB
:1025A000B133BA00FF339858013781880430090AE3
:1025B000023101F0C9FBE8235B00E35CBB42EEDCC7
:1025C000E822F61AED1800235200A354A6E70027CC
:1025D000F1E7200001F090FC00281FD0002E1DDD47
:1025E0007319882647190193B600200001F094FC66
:1025F0005A30800020184068013581880430090A6B
:10260000023101F0A1FB200001F06EFBA359013360
:10261000A351BD4202D0019B9D42E6D1114BE35C28
:10262000002BABD095239B00E35C002BA6D00E4B78
:10263000E15A0029A2D00D4AA35C994202D9013384
:10264000A3549BE700231A212000A35401F0ECFAC5
:1026500094E7C046300DFF1F3409FF1F00140340EC
:10266000E010FF1F5A020000720200005E0200002C
:102670000D4970B54A6E0D4CD2038B69D20BA24244
:1026800006D80B4D0224AA4204D901F075FA70BD98
:1026900002246442E21815007E2425402242F4D030
:1026A000A3432B438B61F0E700F000400A200000B9
:1026B000FC1C0000F8B51D4B1D4F1A78002A10D1E4
:1026C000BA7B002A02D101321A7003E0032AFAD041
:1026D000022AF8D001F0A0FC00220120154B1A704C
:1026E000F8BD154B154D1C68154B9E7801232B70BA
:1026F0002878C0B200F0A2FBBB7B002B0BD101F00D
:10270000CBFAA1239B007343E41883239B00E418B6
:1027100023782B70E4E7032B02D101F0E5FBF0E70F
:102720000020022BDCD101F00FFCEAE71C09FF1F9F
:10273000A60BFF1F2309FF1F3409FF1F490AFF1FB4
:10274000300DFF1FF0B587B00EAD2F780FAD2D788F
:102750000593AC46634614000E4D0CAA12782E78F1
:1027600003930D9B009201932200059B029701F0B9
:102770009BFB2E70012C01D0042C08D1802206492D
:102780008B889343054A1278D20113438B8007B09C
:10279000F0BDC0461C09FF1F6C11FF1F7809FF1F09
:1027A0000B001B3B70B504003020E02B0DD813004C
:1027B000E025493BFF3B9BB2ED00AB4205D8034B04
:1027C000200019825A8201F0C7F970BD8410FF1FE2
:1027D00010B501F0D1FB054B00205B68052B04D937
:1027E000034A5268D20200D4980810BD001000407D
:1027F000FCE100E070B501F0B7F90D4B1B68FC334C
:10280000DC691D6AFFF7E4FF6419844204D2094BB6
:1028100001241B68002B07D004220024064B1A70E9
:10282000064A93690133936101F04EFB200070BDAD
:102830004064FF1F9809FF1F2309FF1FFC0FFF1FA4
:1028400070B50C4D2B68FC335C6A01F08DF9FFF715
:10285000BFFF2B680025FC339B6AE318834204D238
:10286000054B1B68AB4200D1051B01F02DFB280076
:1028700070BDC0464064FF1F9809FF1FD722044B5C
:1028800092009B5810B5002B00D0984710BDC04651
:102890000000FF1F10B501F0D3F8FFF7EFFF274945
:1028A000274BCA6D274C1A4084235B001343CB652A
:1028B000254B1B68186A01F08FF9244B244A1A60D3
:1028C000244B254A1A60A022244B52001A60244B44
:1028D000187801F0B9FB2000224901F085FA0023A5
:1028E000A3600233A360204B2049236003232048C8
:1028F000A36001F079FA10221E4BFF201A6080229B
:1029000052031A60802292031A60802212041A6015
:1029100001F0A2FB012001F0BFFAFA20400001F013
:10292000D3F9582001F038FA134801F04DF901208D
:1029300001F052FA072001F067FB10BD00F00040E3
:1029400000FEFEFF141000404064FF1F0000034023
:102950000180063DBC00034034080000A400034091
:102960004A0AFF1F71020000C3090000FFFF3F0079
:102970002810004000E100E030750000674E336829
:1029800088331B6883F3088801F096F9644A654927
:10299000136800200B401360634B644A1B6893422A
:1029A00000D1A6E001F048FB0221614A13688B4385
:1029B0001360FFF76FFF5F4B5F4C1878C0B201F0F8
:1029C000F3F80023A3600233A3605C4B0120236073
:1029D00001F002F90323A36001F0D6F9040001F02D
:1029E000CBFA050001F0D0F9554B186001F0CCF896
:1029F000544B1968621A531EA14200D21300802260
:102A0000D203934201D39B029B0A3268D16AC90761
:102A100000D471E04C491C0C09689BB24C435943EB
:102A20002402090A641803264849FC3293680A689C
:102A300047489B1A474A0768126847499B18474A04
:102A40009A1833409208DB190A600360042B03D9FB
:102A5000013233400A6003600E684149A619300014
:102A600001F08AF93F4F3E493B68C3183B60300094
:102A7000019301F009FA3C4E30680818384930607B
:102A8000884205D9019B01333B6001F0FDF93160BB
:102A900001F0AAF8354B1B78002B0DD001F06CFA31
:102AA000334B621B196812188A4232D24919091B2A
:102AB000091A304801F098F92F4E337A002B0ED0C6
:102AC00001F05AFA621BF1681218914224D949198F
:102AD000091B091A294801F087F900233372284B92
:102AE00083F3088801F0E0F8002001F0A5FA01F076
:102AF0005BF901F0A1FA5CE7DC0199000234641A89
:102B00005900641A09214B438033CB40A408E418D0
:102B100089E7FA218900CCE71A49DBE74064FF1F07
:102B20001CF00040FFFFC1FF0C0AFF1FB64121034C
:102B300010000040490AFF1F14100040C3090000A4
:102B4000100AFF1F340AFF1F380AFF1F200AFF1F49
:102B5000280AFF1F1C0AFF1F240AFF1FC4090000C8
:102B6000710200006008FF1F2C0AFF1F1C09FF1FD5
:102B7000E408FF1F00100040740BFF1F3C100040D2
:102B800000000020DC050000A022054B92009B58AD
:102B900010B5002B01D0984710BD01F04DF9FBE7AF
:102BA0000000FF1FA122054B92009B5810B5002B7F
:102BB00001D0984710BD01F03FF9FBE70000FF1F6F
:102BC000A222054B92009B5810B5002B01D09847CC
:102BD00010BD01F031F9FBE70000FF1FA322054BF8
:102BE00092009B5810B5002B01D0984710BD01F002
:102BF00023F9FBE70000FF1FA422054B92009B581E
:102C000010B5002B01D0984710BD01F015F9FBE776
:102C10000000FF1F70B501F0AFF94F4B186001F0D5
:102C20008BF80400C30702D401F046F970BD0022FE
:102C30004A4B1A604A4B18780138042829D800F00A
:102C400075FF0320181C2400200001F0B5F80128AE
:102C5000ECD0444C2378042B6ED100F0F5FF002813
:102C6000E4D001F0E1F9582001F096F80223237036
:102C7000DCE7200001F0C0F9E9E7200001F06CF882
:102C8000E5E7200001F050F9E1E7200000F0D4FF73
:102C9000DDE700F0B9FF0500012808D1324B1B78B1
:102CA000053B012B03D82000FFF76EFFD1E72D4B2A
:102CB0001B78022B01D0052B20D1022D28D12B4BC4
:102CC0009B7BAB431CD12000FFF76CFF264B187891
:102CD0000128BED16405BCD4244925224B7B034284
:102CE00005D1233A13405A42534126331A000B7D33
:102CF0009342AED9322000F0C7FFAAE7022D07D1D8
:102D0000194B1B78052B11D12000FFF759FFDDE788
:102D1000012D0BD1012B03D12000FFF75FFF98E7B6
:102D2000062B03D12000FFF767FF92E7200001F098
:102D300083F8022D8DD1C9E7032B04D10C4B987C6D
:102D400001F062F872E7072B00D06FE7094B987B20
:102D500001F062F86AE7C0469C09FF1F9809FF1F4F
:102D60009009FF1F2309FF1F1C09FF1FA60BFF1F50
:102D7000BC0BFF1FD40BFF1FFA210A4B0A4A490064
:102D80001A640A4A5A500A4A04395A50094A083100
:102D90009A64094A5A50094A5C315A50084ADA661C
:102DA0007047C0460000FF1F4527FF1F4128FF1F37
:102DB000F527FF1F2523FF1FB526FF1FC51DFF1F7A
:102DC000991DFF1F10B500F099FE10BDF7B50B0C53
:102DD000FF270122009300233C001E001D009446A3
:102DE000019089B262469A40100008401841361896
:102DF000B6B2FF2F02D1012E00D19FB2009802403F
:102E00001A41AD18ADB2FF2C02D1012D00D19CB2F8
:102E10000133102BE6D10320012E07D1012D04D15F
:102E2000019B2401E4191C700138FEBD102EFCD159
:102E30000238102DF9D00230F7E700008023F7B5F3
:102E40009C46264B264F01932649274A274D284C5E
:102E5000284B02281AD1604638600868264E304058
:102E6000802636033043086001990978002909D18A
:102E70001660224A2A60224A2260E02219689143A1
:102E8000A03A1BE08021C9021160F2E766463E606D
:102E90000F68194E3E408027FF023E430E600199A5
:102EA000097800290DD1176001280ED1154A2A6032
:102EB000154A2260E02219689143C03A0A431A6019
:102EC000F7BD802189021160EEE7E0210F4A02433D
:102ED0002A600F4A22601A688A43F0E74B0AFF1FF4
:102EE000E0000340D800034090000340000003408E
:102EF0005000034040000340FFFFE3FF0280063D17
:102F0000804508220180063D8066082200800698E0
:102F100080550822F8B51E4B80261A680020140040
:102F20003440324232D11A681A4F32431A600122B9
:102F30003B68063093433B6000F04EFE0122164D85
:102F40002B681E432E603B680A2613433B60802794
:102F5000BF00124B1B683B4211D1013EF6B2FF2E5F
:102F600009D17E220E4B1C682B68E40B144093435E
:102F700023432B6005E0082000F02EFEE9E7002E39
:102F8000EFD180222B68600893432B60F8BDC046C8
:102F9000C4F000405CF0004018F0004068F00040D1
:102FA00060F0004010B500F0BFFE01215820034A38
:102FB00001F00AF8FFF7AEFF10BDC046600AFF1F20
:102FC00010B578220021034800F086FE00F014FFBF
:102FD000002010BD4867FF1F70B5040000F0C4FD5D
:102FE00000230C200B4A010059438D18515C002925
:102FF0000DD0A14208D1012300246B7000F084FFA2
:1030000000F062FF200070BD01330A2BEBD11224C7
:10301000F6E7C0464867FF1F70B5040000F0A4FD46
:10302000002319001D000D4A1078002806D0A04288
:103030000CD1557001310C320A29F5D1002B0AD17F
:1030400000F0DAFE00F040FF002070BD5078461E10
:10305000B0411B18EEE700F057FFF3E74867FF1F8A
:10306000F7B504000C20002384460E4D01926746FC
:103070005F43E85D7E19A04212D000280BD10A4BB5
:103080009C4662461B7808331370019B70707C5518
:103090007160B360FEBD01330A2BE8D10320F9E76C
:1030A0000720F7E74867FF1F4467FF1F8020F8B538
:1030B000484BC0051B68C1248360474BFF251A6835
:1030C000012313434361454BA4001A68444B40213C
:1030D0001A60444B1A68444B1A60444B1A59AA436D
:1030E0001A51C52292009E58AE4331438026995012
:1030F0009F583F49F6010F403E439E509E588027FF
:103100003602360A3043985080201A5900020A408D
:1031100002431A5104341A59364E3F043240802675
:103120003A431A511A5936061202120A32431A51F8
:1031300008341A5980260A4002431A51C3229200C9
:103140009F58B446AF4337439F509F58294E0F4076
:1031500007439F509F5837408026360437438026C8
:103160009F509F5836063F023F0A37439F50C02268
:103170001F59AF433A431A511A591202120A164301
:10318000C6221E5192009C58AC4365462C439C506D
:103190009C5800250C4020439850C72080001A58A6
:1031A000154C1140C02212020A431A50134B1B78CF
:1031B000DB08AB4201DC0020F8BD2378002B06D0F1
:1031C000A368002B00D0984701350C34EEE712209D
:1031D000F2E7C0466443FF1F6043FF1FB0F00040AA
:1031E0004067FF1FB4F000403C67FF1F00E100E0B4
:1031F000FF00FFFFFFFF00FF4867FF1F4467FF1F3F
:10320000030010B51F2809D8072200201340072407
:1032100004490A78A24313430B7010BD0023062013
:10322000F5E7C0464467FF1F054B06491B780A684F
:1032300005485B0702401B0B134300200B607047DF
:103240004467FF1F1CF00040FFFFC1FF70B50C2555
:10325000FFF7EAFF0A4B1C780A4BE4086543ED18B8
:10326000002C01D1200070BD2B78002B06D06B689C
:10327000002B00D09847013C0C3DF1E71220F2E70B
:103280004467FF1F3C67FF1F1FB5002102220B0090
:1032900001910091052000F0E7FD02230B490A6827
:1032A0001A42FCD120230393039B5A1E0392002B46
:1032B000FAD1074A1368002BFCDA0B246C44200077
:1032C000012100F0D9FD207804B010BD90C8004065
:1032D00000C8004013B504000A4B0193019B002B6A
:1032E00001D1112016BDFFF7CFFF23000340044298
:1032F00005D0052000F070FC019B013BEDE71800B4
:10330000F0E7C046FFFFFF0707B500F02DFC802265
:103310000821D205936A0191002B01D107399162EE
:1033200002210C4A11600199481E01900029FAD12E
:1033300003311160053101910199481E0190002966
:10334000FAD11160002B02D18022D205936200F0E5
:10335000BBFD07BD00C00040F0B52D4C89B02378FF
:10336000002B4FD1FEF7CEFA02232A4F03903A6882
:103370001A42FCD120230693069B5A1E0692002B6C
:10338000FAD1254E3368002BFCDA0120FFF7A2FFAB
:10339000011E02D0112009B0F0BD030003220190EC
:1033A000009005AD9F2000F05FFD0321280000F094
:1033B00063FD02233A681A42FCD120230793079B3E
:1033C0005A1E0792002BFAD13368002BFCDA012039
:1033D000FFF780FF0028DDD10398FEF7A7FAAA784F
:1033E0006B7811041B020B4329780B4363601300B5
:1033F000113B0A49052B07D801239340A3600B60BA
:10340000012323700020C6E780231B03F6E7C04694
:103410004C43FF1F90C8004000C800409808FF1FA1
:103420001E4B30B55A6818781D4B85B0D3185942D9
:103430004B4101210093002300F0A6FD194B1A4ACD
:1034400002259A6300221A6510325A658022C4212F
:103450009D65164B1648D202DA6789004258154B13
:1034600080241A4080231B041343435064234120CB
:103470000393E40500F006FA402000F003FA6562C9
:10348000039D6B1E0393002DFAD103236362FFF7A4
:103490003BFFA562FFF760FF05B030BD5843FF1F3B
:1034A00095FFFEF700C80040050001FF04E100E0C1
:1034B00000E100E0FFFF00FFF0B585B00700FEF778
:1034C00021FA022305002D4C22681A42FCD1202348
:1034D0000093009B5A1E0092002BFAD1284E3368AD
:1034E000002BFCDA0120FFF7F5FE002803D01124A1
:1034F000200005B0F0BD234B2360022322681A424E
:10350000FCD120230193019B5A1E0192002BFAD17A
:103510003368002BFCDA0120FFF7DCFE0028E6D13F
:10352000194B1F60022322681A42FCD12023029308
:10353000029B5A1E0292002BFAD13368002BFCDA50
:103540000120FFF7C7FE0028D1D1104B23600223D2
:1035500022681A42FCD120230393039B5A1E039234
:10356000002BFAD13368002BFCDA0120FFF7B2FE02
:10357000041EBCD12800FEF7D9F9B9E790C8004075
:1035800000C8004001000006A8C8004001800001FA
:1035900010B50020FFF790FF10BD000010B5064BDE
:1035A00018705960FFF73CFF00211320034AFFF712
:1035B00057FD002010BDC0465843FF1F2134FF1F98
:1035C000F0B5040085B003920291FEF79BF98822C2
:1035D00063035B0B52051A438023DB059D6A80233E
:1035E000274F0092BA68002601901B039A420CD91B
:1035F000F82326001B041E401C4206D08022214BCB
:1036000052025E6219680A431A60002D0BD100F065
:10361000ABFA02221C4B1A608023DB055A62013A86
:103620009A6200F051FC0023039A934220D1002DAE
:103630000AD100F099FA144B03221D608023DB05A8
:103640005A629D6200F040FC8023BA681B039A42D4
:1036500008D9002E06D000220A4B0C495A621A687B
:103660000A401A600198FEF761F9002005B0F0BD2C
:10367000009A0299D2181278CA540133D4E7C0468E
:103680004C43FF1F00C8004000C00040FFFFFEFF8A
:10369000F0B587B0029103920400FEF733F9019070
:1036A00000F062FA802302250122234EDB053560FB
:1036B0005D629A6200F008FC204F3B682B42FCD10F
:1036C00020230493049B5A1E0492002BFAD11C4D14
:1036D0002B68002BFCDA0120FFF7FCFD002802D04C
:1036E000112007B0F0BD2000039A029900F084FA7F
:1036F000022304003A681A42FCD120230593059B5B
:103700005A1E0592002BFAD12B68002BFCDA0120FF
:10371000FFF7E0FD051EE3D100F026FA8023032227
:10372000DB0535605A629D6200F0CEFB0198FEF722
:10373000FDF8E0B2D5E7C04600C0004090C80040A8
:1037400000C80040F0B5802489B00600FEF7DAF822
:10375000E405A36A02250393029000F005FA012311
:10376000304F3D606562A36200F0AEFB2E4C2368D3
:103770002B42FCD120230593059B5A1E0592002B5A
:10378000FAD12A4D2B68002BFCDA0120FFF7A2FDAD
:10379000002803D01124200009B0F0BD244B236081
:1037A000022322681A42FCD120230693069B5A1E4C
:1037B0000692002BFAD12B68002BFCDA0120FFF7D0
:1037C00089FD021EE6D11B4B03211E600300019000
:1037D0000090202000F048FB022322681A42FCD10E
:1037E00020230793079B5A1E0792002BFAD12B68C0
:1037F000002BFCDA0320FFF76DFD041ECAD100F098
:10380000B3F980230322DB053C605A629C6200F01E
:103810005BFB039B002B01D1FFF776FD0298FEF7BF
:1038200085F8B8E700C0004090C8004000C80040DC
:103830000100000694C8004007B50002019104226F
:10384000000A01A9FFF724FF0EBD000073B50500B3
:1038500005240B4AA3005B429B1819686B46DE1DCA
:103860003000FFF7B3FA022804D133782B55013C1E
:10387000EFD276BD052CFCD00128FAD10230F8E752
:10388000140900111F2807D8012380228340D20584
:1038900091680B43936070473F2808D8012380222A
:1038A00020388340D20551690B435361F3E75F2809
:1038B000F1D80123802240388340D205116A0B439E
:1038C0001362E8E71F2807D8012280218240C9053A
:1038D0008B6893438B6070473F2808D80122802172
:1038E00020388240C9054B6993434B61F3E75F2859
:1038F000F1D80122802140388240C9050B6A9343E8
:103900000B62E8E71F2810D880230200DB05153A78
:103910001968012A06D820229143196019680A43C0
:103920001A60704701228240F6E73F2811D88023B1
:103930000200DB05353AD968032A06D810229143E4
:10394000D960D9680A43DA60EBE701222038824067
:10395000F5E75F28E5D842238022181A413B8340CF
:10396000D205516A99435162516A0B435362D8E7B9
:1039700010B50400012813D1A022184992050B6844
:103980005B015B0913430B60154B164A1968114024
:10399000154A0A431A60402219680A431A6010BD8A
:1039A0000028FCD101000A2000F0FEFA21000B20C3
:1039B00000F0FAFAC0220A4B920019680A4340212B
:1039C0001A601A688A431A60B022044912060B680A
:1039D0005B015B0913430B60E1E7C04614F0004054
:1039E0001CF000407F00FEFF80FD010072B6074A18
:1039F0001368013313600422054B1A600023054A43
:103A000013608022D2055360FEE7C0467808FF1F8E
:103A1000C0F00040C4F0004005490B68002B05D100
:103A2000044A0A6004490A60044A13607047C046A9
:103A3000140AFF1F841E0000380AFF1FC4F0004054
:103A40000023034A1360034A1360034A136070475C
:103A500054F0004040F1004044F10040002310B514
:103A6000184C8AB0009301932378012B27D0694624
:103A7000012000F049F9002817D1009B1249029358
:103A8000019B06AA0393114B02A81B680493104BD9
:103A90001B68059300F0A0FA10220E4906A800F05A
:103AA000DBF9002804D1FF23237000200AB010BDE9
:103AB0000123094A074902A8237000F08DFA01206A
:103AC000F4E7C0464464FF1F1029001108290011C3
:103AD0000C290011202900114864FF1F13B501248F
:103AE0006946012000F010F9034B00940193FFF7A1
:103AF000B5FF200016BDC046BB0B000010B5FFF798
:103B00009FFFFFF7EBFF002802D0024B984710BD44
:103B1000FEE7C046E1A2000002B471464908490030
:103B2000095649008E4402BC7047C04602B4714633
:103B300049084900095C49008E4402BC7047C046F0
:103B400003B47146490840004900095A49008E44AF
:103B500003BC70470000000001B40248844601BC69
:103B6000604700BF116E000001B40248844601BCEA
:103B7000604700BF75A9000001B40248844601BC3B
:103B8000604700BFD1AE000001B40248844601BCCA
:103B9000604700BFC166010001B40248844601BC11
:103BA000604700BF6D0B010001B40248844601BCB0
:103BB000604700BF8914010001B40248844601BC7B
:103BC000604700BF8944000001B40248844601BC3C
:103BD000604700BF8D11010001B40248844601BC5A
:103BE000604700BF0189000001B40248844601BC5F
:103BF000604700BFD544010001B40248844601BCBF
:103C0000604700BF9573010001B40248844601BCBF
:103C1000604700BFDD0C010001B40248844601BCCE
:103C2000604700BFE90B010001B40248844601BCB3
:103C3000604700BF53B9000001B40248844601BC8C
:103C4000604700BFF935010001B40248844601BC59
:103C5000604700BF01D7000001B40248844601BCA0
:103C6000604700BF0D52010001B40248844601BC08
:103C7000604700BF51B8000001B40248844601BC4F
:103C8000604700BFE94C010001B40248844601BC12
:103C9000604700BF6137010001B40248844601BC9F
:103CA000604700BFE9F6000001B40248844601BC49
:103CB000604700BF7997000001B40248844601BC08
:103CC000604700BFC9A9000001B40248844601BC96
:103CD000604700BF8512010001B40248844601BC60
:103CE000604700BFB70E000001B40248844601BC23
:103CF000604700BF5976010001B40248844601BC08
:103D0000604700BF2144000001B40248844601BC62
:103D1000604700BFE1AC000001B40248844601BC2A
:103D2000604700BFE927000001B40248844601BC97
:103D3000604700BFED68010001B40248844601BC41
:103D4000604700BFBD0B010001B40248844601BCBE
:103D5000604700BFC115010001B40248844601BCA0
:103D6000604700BF0534010001B40248844601BC2D
:103D7000604700BF85C1000001B40248844601BC11
:103D8000604700BF090E000001B40248844601BC30
:103D9000604700BF156B010001B40248844601BCB6
:103DA000604700BF7912010001B40248844601BC9B
:103DB000604700BF8552010001B40248844601BC3F
:103DC000604700BF0134010001B40248844601BCD1
:103DD000604700BFCD0C010001B40248844601BC1D
:103DE000604700BFE512010001B40248844601BCEF
:103DF000604700BF2D6C010001B40248844601BC3D
:103E0000604700BFADAE000001B40248844601BC6B
:103E1000604700BF4DF9000001B40248844601BC70
:103E2000604700BFC1F7000001B40248844601BCEE
:103E3000604700BFA1B5001101B40248844601BC2F
:103E4000604700BFE917010001B40248844601BC85
:103E5000604700BFB352010001B40248844601BC70
:103E6000604700BFCD4C010001B40248844601BC4C
:103E7000604700BF496D010001B40248844601BC9F
:103E8000604700BF3D71010001B40248844601BC97
:103E9000604700BF090E000001B40248844601BC1F
:103EA000604700BF6911010001B40248844601BCAB
:103EB000604700BF9D6A000001B40248844601BC0F
:103EC000604700BFDD0A010001B40248844601BC1E
:103ED000604700BF9DA9000001B40248844601BCB0
:103EE000604700BF8937010001B40248844601BC25
:103EF000604700BF75F8000001B40248844601BC69
:103F0000604700BF71B0000001B40248844601BCA4
:103F1000604700BF21A9000001B40248844601BCEB
:103F2000604700BFD9B0000001B40248844601BC1C
:103F3000604700BFF535010001B40248844601BC6A
:103F4000604700BF8D82000001B40248844601BC76
:103F5000604700BF19FA000001B40248844601BC62
:103F6000604700BFC1A5000001B40248844601BCFF
:103F7000604700BFE9D4000001B40248844601BC98
:103F8000604700BFC95C010001B40248844601BC1F
:103F9000604700BFC56D010001B40248844601BC02
:103FA000604700BFF9ED000001B40248844601BC3F
:103FB000604700BF1DA2001101B40248844601BC45
:103FC000604700BF8B52010001B40248844601BC27
:103FD000604700BF0167010001B40248844601BC8C
:103FE000604700BFDD3F000001B40248844601BCC9
:103FF000604700BFBD5C010001B40248844601BCBB
:10400000604700BF0934010001B40248844601BC86
:10401000604700BFF90D010001B40248844601BCAD
:10402000604700BFA9D8000001B40248844601BC23
:10403000604700BF6DF6000001B40248844601BC31
:10404000604700BF016C010001B40248844601BC16
:10405000604700BFEDA5000001B40248844601BCE2
:08406000604700BFED6B010099
:104068000200000056BE00110100000068BC0011EB
:104078000200000052BE001101000000A840FF1F0E
:104088000200000070BC001101000000BC61FF1FAD
:104098000200000050BE0011030000003061FF1F45
:1040A800120000000200000056BE001101000000CE
:1040B800B0BC00110200000052BE00110100000057
:1040C800ADBC001102000000BABC001103000000E2
:1040D8006B61FF1F0200000050BE001103000000CA
:1040E8008061FF1F0200000052BE001101000000A5
:1040F800ACBC001102000000B8BC001103000000B5
:104108004161FF1F0200000050BE001103000000C3
:104118006261FF1F0200000056BE0011010000008E
:10412800F0BC00110200000052BE001101000000A6
:10413800F141FF1F0200000002BD00110100000054
:10414800EBBC00110200000052BE0011010000008B
:10415800F041FF1F0200000000BD00110100000037
:104168008861FF1F0200000052BE0011010000001C
:10417800EF41FF1F02000000FEBC0011010000001B
:10418800DBBC00110200000052BE0011010000005B
:10419800EE41FF1F02000000FCBC001101000000FE
:1041A800D6BC00110200000052BE00110100000040
:1041B800ED41FF1F02000000FABC001101000000E1
:1041C800D1BC00110200000052BE00110100000025
:1041D800EC41FF1F02000000F8BC001101000000C4
:1041E800CCBC001102020202020200000000000022
:1041F8000D0C0000C14B0011874B001144BD00118C
:1042080090011D0018001800FFFF070102030405B4
:104218000602010600000000000000000000000087
:104228000000000000000000000000000000000086
:10423800030000000200000056BE0011010000004B
:1042480064BD00110200000052BE00110100000010
:10425800AC42FF1F020000006EBD0011010000000B
:10426800B661FF1F0200000050BE001103000000ED
:104278002064FF1F0200000052BE00110100000070
:10428800AC42FF1F020000006CBD001101000000DD
:10429800B861FF1F0200000050BE001103000000BB
:1042A8001864FF1F126C6C6C00000000005800407E
:1042B800151600000001000000000111FFFF0000BA
:1042C8005048593600000000000000000B000500AF
:1042D800F0000000B4000028002800283075A00075
:1042E800A000A000A00000080008E001F0001000F5
:1042F8001000100010001000100050005000500076
:1043080010001000D0070000000000000F0001009E
:104318000500307507001000010081FF0000000053
:10432800FF000000057400110D7200119D6F00114F
:10433800FFFF0100FF000000219E00119D9B00115E
:10434800B59A0011000000000000000000000800FD
:10435800040000003B0001085902E0018821280000
:10436800FF0000000200000056BE0011010000001E
:104378001CBF00110200000052BE00110100000025
:10438800E943FF1F020000004EBE001101000000BB
:104398000068FF1F0200000052BE0011010000006B
:1043A800E843FF1F020000004CBE0011010000009E
:1043B800E643FF1F0200000052BE0011010000008A
:1043C800E443FF1F020000004ABE00110100000084
:1043D800DC43FF1F180018001D00900102000003B5
:1043E800020200000200000056BE00110100000099
:1043F80030BF00110200000052BE00110100000091
:104408002C44FF1F0200000048BE001100000000FD
:10441800000000000200000050BE00110300000070
:064428002068FF1F20FFC9
:040000051FFF184180
:00000001FF
